:106EC6000000090200000301FA0400EF0500030AAE
:106ED6000A5A0B001E0C00FA0D00030E00040F01E7
:106EE60064100096120132130AFA14010217010AFD
:106EF6001801EF1905321A010A1B01EF1C05321F92
:106F0600FFFF20FFFF23011E2400642A00FA2B0046
:106F1600FA2C50782D003D2E004630006432507811
:106F26003300003432FF35016436016437015038CE
:106F36000A643A00033B00043C00643E003C3F0008
:106F46000140FFFF411450420A5A430AC844053221
:106F56004500B44600FA4900024B00014C00FA50C5
:106F66000C0C510596520A32530B46540A96570595
:106F760046590A465A32FA5B010A5C0A325E000A30
:106F86005F00646200FE64021067FFFF680101692A
:106F960001016A05966B00006C32FF6D00047300F8
:106FA600007400007801327901327E00647FFFFFB1
:106FB60080FFFF8100008400648800028A00019D32
:106FC6000A969E00019FFFFFA0FFFFA2000AA3FFF3
:106FD600FFA40064A50064A6FFFFA7FFFFA8FFFFAC
:106FE600A9FFFF0101241500002F003C470124489A
:106FF60002025602024EFFFF58000261FFFF6600C2
:10700600018500AF8600018700FA89010499000016
:10701600A100FAFAFAFA0065006F00790083008D84
:10702600009700A100AC00B600C000CA00D400DE84
:1070360000E800F2005800600068007000780080E8
:1070460000880090009800A000A800B000B800C119
:1070560000C800D000D800DF00E600EE00F60041D0
:107066000047004D00530059005F0065006C007139
:107076000077007D00830089008F0095009B00A2A9
:1070860000A700AC00B200B900C000C500CA00D21B
:0A70960000D500DD00E100E700EF87
:103D750075A71085F97385FA747E017F00E57412C5
:103D850071B2E5732FFF50010E8E598F5A900024A2
:103D9500E0FCA3E0FDEF2DFDEE3CFC8C5B8D5C9023
:103DA5000044E0FAA3E0FBED2BFBEC3AFA8A5B8BCF
:103DB5005C22E55CF5FBE55BF5FCD29322E55CF561
:103DC500E9E55BF5EAD29422E55CF5EBE55BF5EC1C
:103DD500D29122E55CF5EDE55BF5EED29222E55C4C
:103DE500F5FDE55BF5FED28722E55CF5CEE55BF5F5
:103DF500CFD29022E50C906ABBF82828738052A296
:103E050034B34008E5B54408F5B58006E5B554F783
:103E1500F5B5803DA234B34008E5B54440F5B5801D
:103E250006E5B554BFF5B58028A234B34008E5B51D
:103E35004480F5B58006E5B5547FF5B58013A23409
:103E4500B34008E5B54404F5B58006E5B554FBF582
:013E5500B5B7
:0F6ABB00023E02023E04023E19023E2E023E43FC
:103E560022743390017CF0743690017DF0742D90BD
:103E6600017EF0743290017FF07420900180F0742E
:103E760031900181F07432900182F0744390018395
:103E8600F07479900184F0746C900185F074209040
:103E96000186F07420900187F07420900188F074F8
:103EA60020900189F0742090018AF0229008B3E0F6
:103EB600FEA3E0FF7423D39F74019E400C906EC650
:103EC600120048E493F59980129008B3E0FEA3E04F
:103ED600FF906EC6120048E493F5999008B31271EC
:103EE600C09008B3E0FEA3E0FFEFB45607EEB401BE
:103EF60003754D0022AE59AF5A740A8E048F05FF22
:103F06001271A28C5B8D5CAE59AF5A740A8E048F07
:103F160005FF1271CD8C598D5AE55A4559601374B7
:103F26000AC3955AFFE49559FE8E598F5A785B124B
:103F36007205E573A85BB80015D3955C4010E57370
:103F4600C3955CFFE4955BFE8E5B8F5C8010E5732A
:103F56002424C3955CFFE4955BFE8E5B8F5CAE5BB1
:103F6600AF5C74236F4E600674246F4E701AAE5B9E
:103F7600AF5C74236F4E7005757301800375730211
:103F8600755C22755B008003757300229000B9E0B2
:103F9600B40104C2068002D2069000BAE0B401045D
:103FA600C2078002D2079000F7E075F0E1A4FFAEE9
:103FB600F0740A8E048F05FF1271A29008A7ECF028
:103FC600A3EDF09000F7E075F02BA4FFAEF09000A3
:103FD60020EEF0A3EFF07E017F009000B5E01271B5
:103FE600B29000F8E08E048F05FF1271A2740AFFEA
:103FF6001271A28D60900101E075F0E1A4FFAEF0B0
:10400600740A8E048F05FF1271A29008ABECF0A320
:10401600EDF0900103E06013900103E0F5F07416F3
:1040260084FF7E00EF900909F08006746490090908
:10403600F09000F9E0900097F0900147E0FE9000C4
:10404600F5E08E0088F0A4FFAEF0EF900912F09034
:104056000120E075F013A4FDACF0900044ECF0A351
:10406600EDF0A221B34016900191E0700C90019200
:10407600E07006900193E060028002C221900191F7
:10408600E0B4300F900192E0B44708900193E064E9
:104096003B60028004D2228002C2229000B2E0FE7F
:1040A600900913E06E601B7599E612019C74AB9043
:1040B6000071F01206DA7464F50975080012062418
:1040C60080FE9000AAE0700674009000DFF0900079
:1040D6009BE0FE9000DFE0B5063F90009DE0FE907D
:1040E60000FDE0B5063390009CE0FE90010BE0B5C4
:1040F600062790009EE0FE9000B2E0B5061B9000F9
:104106009FE0FE90012BE0B5060F9006ECE0FE90D6
:1041160000A0E06E700302427A740790012EF090C0
:1041260000B2E0B4010674009000B2F09000B2E074
:10413600B4020674009000FDF09000B2E0B40306ED
:10414600740090010AF090010BE0B401277400900E
:1041560000C7F0741C900131F074009006F3F074FF
:10416600009006F4F09000DFE0B4020674019000BF
:10417600DFF080339000DFE0B4021A741C9000C7B1
:10418600F07400900131F074009006F3F074009022
:1041960006F4F080127400900131F074009000C7AC
:1041A600F0741C9006F3F09000FDE0D394014026D5
:1041B60074009000C6F0741B900130F074009006F5
:1041C600EFF074009006F0F09000DFE060067400F7
:1041D6009000DFF080329000DFE0601A741B9000E0
:1041E600C6F07400900130F074009006EFF0740091
:1041F6009006F0F0801274009000C6F074009001F2
:1042060030F0741B9006EFF09006ECE06008740046
:104216009007A3F0800674299007A3F09000D2E0DF
:1042260060147409900135F074009006F7F074007C
:104236009006F8F0800C7400900135F07409900631
:10424600F7F0D2209000DFE090009BF090010BE0A9
:1042560090009CF09000FDE090009DF09000B2E090
:1042660090009EF090012BE090009FF09006ECE00D
:104276009000A0F09000A1E0FE9000D2E06E603EBB
:104286009000D2E0600E7409900135F0740090063B
:10429600F7F0800C7400900135F074099006F7F081
:1042A6009000A1E060069000D2E07002D22090005B
:1042B600D2E09000A1F09000D2E09008BDF090010D
:1042C60015E0B40117900030740FF0A374FFF0905E
:1042D6000032E4F0A3F07402900115F0900115E0AD
:1042E600B40341900032E0FEA3E0FF900030E0FC12
:1042F600A3E0FD1271FD74101271B2740812003938
:10430600EF900114F0EF700674FF900114F0740042
:10431600900115F0900031E09000CBF0900030E075
:104326009000CCF09000A6E09000A3F09000A5E0ED
:104336009000A2F09000D4E0C3941E50569000D492
:10434600E0F404241E9000A4F09000A4E075F00AA6
:1043560084FF7E008F739000A4E075F00A84ADF0B0
:104366007C008D749000A2E0D39574400D9000A25D
:10437600E0C395749000A2F0800F9000A2E0240A9A
:10438600C395749000A2F005739000A3E025739086
:1043960000A3F09000A3E090005EF090005EE0D3F2
:1043A6009424400B90005EE0C3942490005EF0904D
:1043B600005EE0240690005FF090005EE0240C9022
:1043C6000060F090005EE02412900061F090005EC4
:1043D600E02418900062F090005EE0241E900063D6
:1043E600F090005FE0D39424400B90005FE0C3940C
:1043F6002490005FF0900060E0D39424400B90007E
:1044060060E0C39424900060F0900061E0D39424AF
:10441600400B900061E0C39424900061F09000622C
:10442600E0D39424400B900062E0C3942490006291
:10443600F0900063E0D39424400B900063E0C394B3
:1044460024900063F090006AE4F090005EE064233C
:10445600600790005EE0B4242090005EE0B423067E
:10446600740290006AF090005EE0B4240690006A40
:104476007401F090005E7401F090006BE4F090001F
:104486005FE06423600790005FE0B4242090005F43
:10449600E0B42306740290006BF090005FE0B42451
:1044A6000690006B7401F090005F7401F090006C50
:1044B600E4F0900060E064236007900060E0B424BC
:1044C60020900060E0B42306740290006CF0900027
:1044D60060E0B4240690006C7401F09000607401F2
:1044E600F090006DE4F0900061E0642360079000B6
:1044F60061E0B42420900061E0B4230674029000C9
:104506006DF0900061E0B4240690006D7401F090A7
:1045160000617401F090006EE4F0900062E06423A4
:104526006007900062E0B42420900062E0B42306A5
:10453600740290006EF0900062E0B4240690006E63
:104546007401F09000627401F090006FE4F0900046
:1045560063E064236007900063E0B4242090006366
:10456600E0B42306740290006FF0900063E0B42478
:104576000690006F7401F09000637401F09000A63D
:10458600E0FE900109E02E900072F0900072E06467
:10459600126007900072E0B42406900072E004F006
:1045A600900072E064116007900072E0B4230690F8
:1045B6000072E014F0900072E0D39424400B900057
:1045C60072E0C39424900072F0900072E0D39412CB
:1045D600400D900072E0C39412900073F0800A9030
:1045E6000072E02412900073F0755D129000A6E050
:1045F600FE9000ECE0D39E50139000A6E0FE9000E3
:10460600ECE0F4042E04900064F080139000A6E021
:104616002424FE9000ECE0F4042E04900064F09054
:104626000064E075F00684AFF07E00EF4E700690F1
:104636000064E004F0900064E00475F00684AFF0D6
:104646007E00EF4E7006900064E014F0900064E087
:10465600B425069000647401F0900064E02406908E
:104666000065F0900064E0240C900066F090006411
:10467600E02412900067F0900064E024189000682F
:10468600F0900064E0241E900069F0900065E0D38D
:104696009424400B900065E0C39424900065F0904C
:1046A6000066E0D39424400B900066E0C394249007
:1046B6000066F0900067E0D39424400B900067E01A
:1046C600C39424900067F0900068E0D39424400BD4
:1046D600900068E0C39424900068F0900069E0D3ED
:1046E6009424400B900069E0C39424900069F01272
:1046F600019C22C293C294C291C292C287C290E523
:10470600B554EFF5B5E5B554DFF5B5C296C295C219
:10471600A0C297C2A2C2A1E5B554BFF5B5E5B5548E
:104726007FF5B5E5B554FBF5B5C208755E46900054
:10473600EFE07005756D028003756D0375540075A5
:10474600530090001874FFF0A374DCF0C20EC21080
:10475600C212C214C216C21874C8900046F074C8B9
:1047660090004AF074C890004EF074C8900052F061
:1047760074C8900056F074C890005AF075520075CF
:104786005100C203754600E56FB41303756F0075DB
:104796006300900026E4F0A3F0757010C20BC20C03
:1047A600C20DC20275560075550090001AE4F0A3BA
:1047B600F090001CE4F0A3F0C22475580075570071
:1047C6009000B1E075F032A4FFAEF090002EEEF04E
:1047D600A3EFF090090FE4F022755A00755900AE68
:1047E60059AF5A7422C39F74019E50030248D39056
:1047F6006EC6120048E493645F6023906EC6120092
:1048060048E493647E6017906EC6120048E4936491
:1048160081600B906EC6120048E493B4840302488C
:10482600B3AE59AF5A906EC6120048E4939000A5F5
:104836001271E30FBF00010EE0FC906EC612004835
:10484600ECFEE493FFEEC39F5026AE59AF5A0FBF5E
:1048560000010E906EC6120048AE59AF5AE493FCA2
:10486600906EC6120048E4939000A51271E3ECF036
:10487600AE59AF5A906EC6120048E4939000A51246
:1048860071E3E0FC906EC8120048ECFCE493FDEC8A
:10489600D39D4019906EC8120048E493FC906EC6F2
:1048A600120048E4939000A51271E3ECF0AE59AF04
:1048B6005A74022FFF50010E8E598F5A785A74017E
:1048C60026F6500418E436F640030247E522755AE8
:1048D60000755900AE59AF5A7432BE00039F50039B
:1048E6000249A1906FE9120048E4939000A5127165
:1048F600E30FBF00010EE0FC906FE9120048ECFEEA
:10490600E493FFEEC39F5026AE59AF5A0FBF000186
:104916000E906FE9120048AE59AF5AE493FC906FBF
:10492600E9120048E4939000A51271E3ECF0AE5949
:10493600AF5A906FE9120048E4939000A51271E314
:10494600E0FC906FEB120048ECFCE493FDECD39D89
:104956004019906FEB120048E493FC906FE9120047
:1049660048E4939000A51271E3ECF0AE59AF5A7487
:104976002D6F4E7006755A33755900AE59AF5A747D
:10498600022FFF50010E8E598F5A785A740126F65F
:10499600500418E436F640030248DA2275A710855B
:1049A600F97385FA747E017F00E5741271B2E573BE
:1049B6002FFF50010E8E598F5AAC5BAD5CEF2DFD6B
:1049C600EE3CFC8C5B8D5CD293D294D291D292D287
:1049D60087D290E55CF5FBE55BF5FCE55CF5E9E582
:1049E6005BF5EAE55CF5EBE55BF5ECE55CF5EDE53D
:1049F6005BF5EEE55CF5FDE55BF5FEE55CF5CEE524
:104A06005BF5CF75A7002285F97385FA747E017F61
:104A160000E5741271B2E5732FFF50010E8E598FA7
:104A26005A7E017F7690012AE01271B2AC59AD5AD6
:104A3600ED2FFFEC3EFE8E5B8F5CE55CF5E9E55BFA
:104A4600F5EA900097E4F07412900075F02285F96B
:104A56007385FA747E017F00E5741271B2E5732FD7
:104A6600FF50010E8E598F5A900020E0FCA3E0FD06
:104A7600EF2DFDEE3CFC8C5B8D5CE55CF5FBE55BB0
:104A8600F5FC22056422A2D9B340089000F9E09013
:104A96000097F0A2D8B3400CC296C295C2A0C297A6
:104AA600C2A2C2A175D8402285A77275A710A2D846
:104AB600B34002C293A2D9B34002C294A2DAB34071
:104AC60002C291A2DBB34002C292A2DCB34002C290
:104AD60087A2DDB34002C29075D8408572A72290A6
:104AE600F800E4936406600280FE12009E75A7003B
:104AF60075D80075D90475DA0975DB0975D840755E
:104B0600A71075D80075D90475DA0975DB0975DC47
:104B16000975DD0975DE0975DF0975D84075A700C9
:104B26001200FB74C8F50975080012062475A70F54
:104B3600E5FC900084F0E5FB900085F0E5FA900036
:104B460086F0E5F9900087F075A70090F800E493E9
:104B5600F5271207439008BCE0D39403500790084A
:104B6600BCE0B4010674009008BCF09008BCE0906C
:104B76000913F074019000EEF09008BCE0906ACA48
:104B8600F8282873802A802875A70F75F30F75A754
:104B960000A2A3400674029000EEF0801375A70FE2
:104BA60075F31775A700A2A4400674029000EEF0F4
:0C6ACA00024B8A024B8C024B8E024BA345
:104BB6009000EEE0B4022AC21C120AEC74029000C5
:104BC600EEF09008BCE0906AD6F828287380108032
:0F4BD6000E74009000FDF08006740090010AF04C
:0C6AD600024BD3024BD5024BD7024BDF22
:104BE5008028D21C120A0174019000EEF09008BCD6
:104BF500E0906AE2F82828738010800E7400900017
:0A4C0500FDF08006740090010AF033
:0C6AE200024BFD024BFF024C01024C096C
:104C0F0090F807E493900091F0900091E0440890A1
:104C1F000091F0900091E054FE900091F01203BDCE
:104C2F00123E579008C9E0900191F09008CAE090A9
:104C3F000192F09008CBE0900193F0900191E07019
:104C4F000C900192E07006900193E060028004C224
:104C5F00218002D2219000DFE00490009BF09000B1
:104C6F00D2E0049000A1F0900149E0B4FF06740077
:104C7F00900149F090014AE0B4FF06740090014A98
:104C8F00F01247DF1248D47400900115F0123F92D2
:104C9F00E5B54401F5B57406900077F07400900007
:104CAF0078F07401900079F090F802E49390007A14
:104CBF00F090F803E49390007BF090F804E4939065
:104CCF00007CF0740690007DF0743B90007EF074D1
:104CDF000390007FF07407900080F07401900081C2
:104CEF00F090F805E493900082F090F806E493902A
:104CFF000083F0740090008BF0740090008CF074BF
:104D0F000090008DF0740090008EF0740090008F72
:104D1F00F07400900090F074FF900092F0A2B6B380
:104D2F009204A2B3B39205A2A4B3921EA2A3B3920C
:104D3F001F900093E4F0756F00743A9007A5F0741C
:104D4F00FD9007A6F0900094E4F0756E0190007549
:104D5F00E4F09000EFE0B40106741A900075F0C211
:104D6F001D756300C209D20AC202757100C22012FA
:104D7F0005C6755F00756B007561007565327566E8
:104D8F0000756700756800756900756A00900026E8
:104D9F00E4F0A3F0756C00D2B2D2A4D2B0D2B1D2EB
:104DAF00A3D2A7D2A6D2A5D2B77E017F009000CC06
:104DBF00E01271B29000CBE02FFF50010E90003047
:104DCF00EEF0A3EFF0EFD394FFEE940F40079000B7
:104DDF0030E4F0A3F0900114E0700674FF9001141A
:104DEF00F09000EFE07005756D028003756D037430
:104DFF0007900132F07408900133F0742A90013457
:104E0F00F074299006EBF07415900793F0741690D8
:104E1F000794F07417900795F07418900796F07434
:104E2F0019900797F0741A900798F07400900799EB
:104E3F00F0740090079AF0740190079BF074029041
:104E4F00079CF0740390079DF0740490079EF07414
:104E5F000590079FF074069007A0F074009007A1CB
:104E6F00F074009007A2F0D29CE570D39410400329
:104E7F007570109006ECE0D3940C40067400900609
:104E8F00ECF09006F0E0D3940C400674009006F01E
:104E9F00F09006F4E0D3940C400674009006F4F002
:104EAF009006F8E0D3940C400674009006F8F0D208
:104EBF00EC75CF01A298B34005C298120C54E54D82
:104ECF006006A299B3B340028005C2991210E0E5C3
:104EDF004E64016005E54EB4040280D5C28E7E108B
:104EEF007F00E5641271B2E58D75F010A4FDACF092
:104EFF00EF2DFDEE3CFCE58B75F01084FF7E00ED91
:104F0F002FFFEC3EFE8E538F54D28E9000D2E06076
:104F1F00099000D2E0C3943D4002805690002812C1
:104F2F0071C0900028E0FEA3E0FF90002AE0FCA3F0
:104F3F00E0FDEFB5053CEEB50438B21AA203B3405D
:104F4F0013A21AB34008E5B54404F5B58006E5B5DC
:104F5F0054FBF5B590002AE0FEA3E0FF90002CE093
:104F6F00FCA3E0FDEF2DFDEE3CFC90002AECF0A33E
:104F7F00EDF09000DFE060099000DFE0C3940340A4
:104F8F00028077123027A20340089000C9E0F54550
:104F9F00801BE55FC395605005754500800F90003D
:104FAF00B6E0C3956150069000DCE0F545E5457528
:104FBF00F002A4FFAEF09008B1EEF0A3EFF0AC2E2C
:104FCF00AD2FEDD39FEC9E4015E5B554BFF5B590D1
:104FDF0000DFE0B40206E5B54480F5B5801C900013
:104FEF0093E0C3942E5013E5B54440F5B59000DF20
:104FFF00E0B40206E5B5547FF5B59000DFE0B403E9
:10500F0024123142AE2EAF2F9008B1E0FCA3E0FD89
:10501F00EFD39DEE9C4008E5B54440F5B58006E51D
:10502F00B554BFF5B5A2B6300401B35003025617FD
:10503F00A2B6300401B35003025617A2B6300601D0
:10504F00B350030254F9756E009000D2E0B43D13D3
:10505F00A206B34008E5B554FBF5B58006E5B544A7
:10506F0004F5B5055EA208B3B35013AE53AF549019
:10507F000018E0FCA3E0FDEDC39FEC9E400302513E
:10508F00ABE56DB4032EA224B34022E55EB4230337
:10509F00756D01E55EC3942350069000757401F0A1
:1050AF00E55ED3942340067402900075F0755E019F
:1050BF00D2248062E56DB40206756D01755E23E53D
:1050CF005EB42305755E01804D900075E07038E584
:1050DF005EC3942350069000757401F0E55ED3947F
:1050EF002340067402900075F0E55EC394235002CE
:1050FF00D21DE55ED394234002D21DC296C295C243
:10510F00A0C297C2A2C2A19000EFE0B4010512465F
:10511F00F98003755E01AE55AF56AC53AD54EF2D0C
:10512F00FDEE3CFC74028C068D071200398E558FF4
:10513F00569000D2E060099000D2E0C3943D400247
:10514F008043900028E0FEA3E0FF9000D2E08E04A1
:10515F008F05FF1271A274018C068D071200399012
:10516F00002CEEF0A3EFF090002CE0F8A3E09000FD
:10517F002AC8F0A3C8F0900028E4F0A3F0C21AE503
:10518F00B554FBF5B5A2A4B34002C21EA2A3B3400F
:10519F0002C21FA21DB34002C21D803AAE55AF56C8
:1051AF00AC53AD54EF2DFDEE3CFC74018C068D0716
:1051BF001200398E558F56E56DC39402500DAC53C6
:1051CF00AD547488C39D74139C400280091246F934
:1051DF007406900075F0E55EB423127403900075A9
:1051EF00F0D21D9000EFE0B401031246F9AE57AFB5
:1051FF0058AC53AD54EF2DFDEE3CFC8C578D58AE93
:10520F0053AF54EFD39DEE9C401190001EE0FAA3D4
:10521F00E0FBEBC394E8EA94034002800690001E83
:10522F001271C090001CE0FEA3E0FFAC53AD54EF31
:10523F002DFDEE3CFC90001CECF0A3EDF09000EF88
:10524F00E0B40118AE53AF5474051271B274011269
:10525F000039900018EEF0A3EFF08011AE53AF5469
:10526F0074021271B2900018EEF0A3EFF0C28E75B7
:10527F008D00758B00756400755401755300D28EC7
:10528F00E55E240875F00984AFF07E00EF4E6003F1
:10529F00025324E56D6013AE55AF5674091271B207
:1052AF0090001AEEF0A3EFF0800F90001CE0F8A32F
:1052BF00E090001AC8F0A3C8F090001AE0FEA3E037
:1052CF00FFEF4E600B7C837D901270A08E518F523A
:1052DF0090001CE4F0A3F0AE51AF527428BE00034F
:1052EF009F5010E5632FFF50010E74011200398E8D
:1052FF00518F528552639000F6E0A851B8000DD33C
:10530F0095524008E552900074F080099000F6E045
:10531F0014900074F0E55E640B6005E55EB41D0942
:10532F009000DFE06003122CDD900072E0655E609C
:10533F0007900073E0B55E03756F00A209B35006C6
:10534F00A208B3B340030253FD9000ABE0B4017366
:10535F0090012DE0B40214121281900098E075F0C4
:10536F00BCA4FFAEF08E5B8F5C8056E56775F00ACC
:10537F0084FF7E009005A5120048E0F55A7559008C
:10538F00AE59AF5A9000D0E01271B274648E048F90
:10539F0005FF1271A28C5B8D5CE55C900070F0AE26
:1053AF0059AF5A9000A9E01271B274648E048F0540
:1053BF00FF1271A274BC8C068D071271B28E5B8FB7
:1053CF005C80179000A9E075F0BCA4FFAEF08E5B77
:1053DF008F5C9000D0E0900070F0E561C394CC50EA
:1053EF0006E55C455B700280031249A2D209E56DA8
:1053FF00B40106E55E640B6002800C7570009000CE
:10540F00767401F0756D00E56D60030254F4900041
:10541F00F2E0600D900097E0A851B8000695524059
:10542F000280589000F2E0B4023790005EE0655EB3
:10543F00602790005FE0655E601F900060E0655E32
:10544F006017900061E0655E600F900062E0655E3E
:10545F006007900063E0B55E03757003756C0080A4
:10546F000CC200756C00900026E4F0A3F09000973A
:10547F00E060067409900075F0806A90005EE0B5F8
:10548F005E0B7570009000767401F0805890005F8D
:10549F00E0B55E0B7570007402900076F080469058
:1054AF000060E0B55E0B7570007403900076F080BD
:1054BF0034900061E0B55E0B757000740490007657
:1054CF00F08022900062E0B55E0B7570007405905D
:1054DF000076F08010900063E0B55E09757000747F
:1054EF0006900076F0A206B39204A206B330B6017E
:1054FF00B35003025617756E019000D2E0B43D13FE
:10550F00A206B34008E5B54404F5B58006E5B554E9
:10551F00FBF5B5E5B54401F5B5741F900093F0A206
:10552F00069204E55ED3944A4014D208E55ED39404
:10553F006D400B7405900075F0D21D755E4690019D
:10554F0028E0A851B80005D39552500D900127E0DF
:10555F00A851B80004955250028008E5B54402F5F1
:10556F00B58017900129E0D395614008E5B5440255
:10557F00F5B58006E5B554FDF5B59000FAE0B40138
:10558F0007E56AC3944140028018E56AC39414503A
:10559F00087413900075F08006740E900075F01269
:1055AF0046F990007DE0FE90007AE0C39E4009909E
:1055BF00007AE0D39408400974FB900075F012460E
:1055CF00F990007BE0601590007BE0FE900079E0A1
:1055DF006E600974FC900075F01246F990007CE043
:1055EF00601590007CE0FE90007EE06E600974FE16
:1055FF00900075F01246F99008BCE0600690012A01
:10560F00E060028003120BD7A21DB3400CC296C2FA
:10561F0095C2A0C297C2A2C2A190012AE0600CAEAF
:10562F0051AF527414BE00059F400280379000B2F4
:10563F00E0906AEEF8282873802A8028A2A3B3503E
:10564F0005A21FB340028005124A0DD21F8015A27A
:10565F00A4B35005A21EB340028005124A0DD21EFC
:04566F008002800035
:106AEE0002564702564902564B02565E0256710234
:026AFE005673CD
:10567300A20BB3B35008900064E0655E600280360D
:10568300A201B35006A200B3B340028023123D75BA
:10569300123DB790010BE0B40113A202B34008E539
:1056A300B54480F5B58006E5B5547FF5B575A7001B
:1056B300C20BD20CD20DA20CB3B35008900065E01C
:1056C300655E60028036A201B35006A200B3B34008
:1056D300028023123D75123DC290010BE0B4011309
:1056E300A202B34008E5B54480F5B58006E5B5549C
:1056F3007FF5B575A700D20BC20CD20DA20DB3B3C3
:105703005008900066E0655E60028036A201B350E7
:1057130006A200B3B340028023123D75123DCD9023
:10572300010BE0B40113A202B34008E5B54480F5D0
:10573300B58006E5B5547FF5B575A700D20BD20C3D
:10574300C20DA20BB3B35008900067E0655E600220
:105753008036A201B35006A200B3B34002802312E5
:105763003D75123DD890010BE0B40113A202B34082
:1057730008E5B54480F5B58006E5B5547FF5B57504
:10578300A700C20BD20CD20DA20CB3B350089000E9
:1057930068E0655E60028036A201B35006A200B3E2
:1057A300B340028023123D75123DE390010BE0B438
:1057B3000113A202B34008E5B54480F5B58006E5C0
:1057C300B5547FF5B575A700D20BC20CD20DA20D4F
:1057D300B3B35008900069E0655E60028036A201B1
:1057E300B35006A200B3B340028023123D75123DAD
:1057F300EE90010BE0B40113A202B34008E5B544F7
:1058030080F5B58006E5B5547FF5B575A700D20BD5
:10581300D20CC20DE570906B00F82828739001122A
:01582300E0A4
:036B000002582018
:10582400906B33F828287312260C801212260C80F1
:0E5834000D122696800812274280031227428A
:0F6B330002582B02583002583502583A02583F88
:10584200757001025EF012286E12298575700202CF
:105852005EF0122D21A203B340139000F7E075F021
:105862001DA4FFAEF0900020EEF0A3EFF09008A58B
:10587200E0FEA3E0FF740A1271B290001AE0FCA3EA
:10588200E0FD74098F02FF1271A28D078C038E0452
:105892008A058B061270A09008A9EEF0A3EFF074AF
:1058A200F0BE00039F500B74F09008A9F8E4F0E8F2
:1058B200A3F0E53670037536019008A9E0FEA3E077
:1058C200FFE5362FFF50010E9008A9EEF0A3EFF08E
:0B58D200757003A22B4029900076E0C7
:066B03000258480258543C
:1058DD00906B42F8282873801C75700A80177570BC
:1058ED000B801275700C800D75700D800875700E23
:0558FD00800375700F2F
:106B42000258E40258E60258EB0258F00258F502E5
:056B520058FA0258FF93
:10590200025EF09006ECE06006750801122E4FA2CE
:105912002DB3B350089007A3E0642960028009E523
:10592200B54408F5B50259CB9000E0E0D3940240AB
:10593200459000B4E02403A851B8000495525009E0
:105942009000B6E0D395615002800ED201A22340AE
:10595200067408900075F0D2239000B4E0A851B804
:105962000005D39552500B9000B6E02403C3956115
:105972005002C20180539000B4E02403A851B80041
:105982000495525010E55FC3956050099000B6E04F
:10599200D395615002800ED201A223400674089072
:1059A2000075F0D2239000B4E0A851B80005D39559
:1059B200525014E560240FC3955F400B9000B6E08F
:1059C2002403C395615002C201A2014002C223A274
:1059D2002DB3500DA201B350089007A3E0642960D3
:1059E200028006E5B554F7F5B59000FAE07007E5D8
:1059F2006AC3941440028002D2019000EFE0B40125
:105A020002D201A2014005757004800A75701090DF
:0D5A12000026E4F0A3F0025EF09000E0E05A
:066B0900025905025A1BAF
:105A1F00906B57F8282873121397801212139780E0
:0E5A2F000D12154A800812160180031216018E
:0F6B5700025A26025A2B025A30025A35025A3A73
:105A3D009006F0E06006750802122E4F7570050293
:105A4D005EF012175A7570069006F4E06006750840
:105A5D0003122E4F025EF0900070E06006A203B3B9
:105A6D00B34002800DE55ED394065006900070E0C1
:105A7D0014F01219E37570079006F8E060067508CA
:105A8D0004122E4F025EF090012DE0B402031213AA
:105A9D0008121E4B757008025EF0121F2D757009ED
:105AAD00025EF0122305A20BB35005A20CB3400207
:105ABD008006D20BD20CD20D757010025EF09000E4
:105ACD0048E0C394465008C2967446900048F09042
:105ADD00006AE0B4011DE536240AF5369008A9E008
:105AED00FEA3E0FF740A2FFF50010E9008A9EEF0FF
:105AFD00A3EFF090006AE0B4021DE5362414F536EC
:105B0D009008A9E0FEA3E0FF74142FFF50010E9042
:105B1D0008A9EEF0A3EFF085365A75590090005E96
:105B2D00E0F573123EFBE55C900048F090000CE54B
:105B3D0059F0A3E55AF0E573900049F0C20F9008B3
:105B4D00A9E0F559A3E0F55A90005EE0F573123E19
:105B5D00FBE55C900046F0900000E559F0A3E55A96
:105B6D00F0E573900047F0C20E757003025EF09081
:105B7D00004CE0C394465008C295744690004CF01A
:105B8D0090006BE0B4011DE536240AF5369008A9A6
:105B9D00E0FEA3E0FF740A2FFF50010E9008A9EE5E
:105BAD00F0A3EFF090006BE0B4021DE5362414F580
:105BBD00369008A9E0FEA3E0FF74142FFF50010EEC
:105BCD009008A9EEF0A3EFF085365A7559009000B4
:105BDD005FE0F573123EFBE55C90004CF090000E1B
:105BED00E559F0A3E55AF0E57390004DF0C2119020
:105BFD0008A9E0F559A3E0F55A90005FE0F573129E
:105C0D003EFBE55C90004AF0900002E559F0A3E5FB
:105C1D005AF0E57390004BF0C210757003025EF000
:105C2D00900050E0C394465008C2A07446900050B6
:105C3D00F090006CE0B4011DE536240AF5369008AD
:105C4D00A9E0FEA3E0FF740A2FFF50010E9008A9F2
:105C5D00EEF0A3EFF090006CE0B4021DE5362414D5
:105C6D00F5369008A9E0FEA3E0FF74142FFF500154
:105C7D000E9008A9EEF0A3EFF085365A75590090F5
:105C8D000060E0F573123EFBE55C900050F0900073
:105C9D0010E559F0A3E55AF0E573900051F0C213E9
:105CAD009008A9E0F559A3E0F55A900060E0F5736E
:105CBD00123EFBE55C90004EF0900004E559F0A318
:105CCD00E55AF0E57390004FF0C212757003025E55
:105CDD00F0900054E0C394465008C297744690006B
:105CED0054F090006DE0B4011DE536240AF53690B0
:105CFD0008A9E0FEA3E0FF740A2FFF50010E9008E3
:105D0D00A9EEF0A3EFF090006DE0B4021DE536248E
:105D1D0014F5369008A9E0FEA3E0FF74142FFF5090
:105D2D00010E9008A9EEF0A3EFF085365A755900D3
:105D3D00900061E0F573123EFBE55C900054F0902D
:105D4D000012E559F0A3E55AF0E573900055F0C245
:105D5D00159008A9E0F559A3E0F55A900061E0F51A
:105D6D0073123EFBE55C900052F0900006E559F091
:105D7D00A3E55AF0E573900053F0C2147570030259
:105D8D005EF0900058E0C394465008C2A27446904D
:105D9D000058F090006EE0B4011DE536240AF5368A
:105DAD009008A9E0FEA3E0FF740A2FFF50010E90AA
:105DBD0008A9EEF0A3EFF090006EE0B4021DE536F9
:105DCD002414F5369008A9E0FEA3E0FF74142FFF0C
:105DDD0050010E9008A9EEF0A3EFF085365A7559D3
:105DED0000900062E0F573123EFBE55C900058F008
:105DFD00900014E559F0A3E55AF0E573900059F0C1
:105E0D00C2179008A9E0F559A3E0F55A900062E099
:105E1D00F573123EFBE55C900056F0900008E559D5
:105E2D00F0A3E55AF0E573900057F0C216757003B4
:105E3D00025EF090005CE0C394465008C2A1744627
:105E4D0090005CF090006FE0B4011DE536240AF57A
:105E5D00369008A9E0FEA3E0FF740A2FFF50010E53
:105E6D009008A9EEF0A3EFF090006FE0B4021DE5ED
:105E7D00362414F5369008A9E0FEA3E0FF74142F24
:105E8D00FF50010E9008A9EEF0A3EFF085365A757C
:105E9D005900900063E0F573123EFBE55C90005CE9
:105EAD00F0900016E559F0A3E55AF0E57390005D0A
:105EBD00F0C2199008A9E0F559A3E0F55A900063D6
:105ECD00E0F573123EFBE55C90005AF090000AE598
:105EDD0059F0A3E55AF0E57390005BF0C2187570A8
:035EED000380002F
:106B0F00025A4F025A64025A94025AA7025AB0020A
:106B1F005ACB025B7C025C2D025CDE025D8F025E53
:046B2F0040025EF0D2
:105EF000900046E0B55E028003025F92A20E4072FF
:105F0000900000E0FEA3E0FFEF4E6021AE55AF56DB
:105F1000900000E0FCA3E0FD120003740A8E048FE1
:105F200005FF1271A2900000ECF0A3EDF090004785
:105F3000E0601A900000E0FEA3E0FFAC55AD56EF24
:105F40002DFDEE3CFC900000ECF0A3EDF09000473E
:105F5000E0D39401401A900000E0FEA3E0FFAC55AE
:105F6000AD56EF2DFDEE3CFC900000ECF0A3EDF003
:105F7000D20EAE53AF54900000E0FCA3E0FDEFC39F
:105F80009DEE9C400D124A54D296C20E74C89000E9
:105F900046F0A20EB3B35007900046E0B55E028013
:105FA0000D124A54D29674C8900046F0C20E90006A
:105FB00048E0B55E02800302604DA20F407290007F
:105FC0000CE0FEA3E0FFEF4E6021AE55AF5690000F
:105FD0000CE0FCA3E0FD120003740A8E048F05FFA1
:105FE0001271A290000CECF0A3EDF0900049E0607B
:105FF0001A90000CE0FEA3E0FFAC55AD56EF2DFD6E
:10600000EE3CFC90000CECF0A3EDF0900049E0D3E6
:106010009401401A90000CE0FEA3E0FFAC55AD5691
:10602000EF2DFDEE3CFC90000CECF0A3EDF0D20F58
:10603000AE53AF5490000CE0FCA3E0FDEFC39DEE27
:106040009C400AC2967446900048F0C20FA20FB35B
:10605000B35007900048E0B55E02800AC2967446CD
:10606000900048F0C20F90004AE0B55E0280030243
:106070006108A2104072900002E0FEA3E0FFEF4E24
:106080006021AE55AF56900002E0FCA3E0FD120087
:1060900003740A8E048F05FF1271A2900002ECF0C7
:1060A000A3EDF090004BE0601A900002E0FEA3E048
:1060B000FFAC55AD56EF2DFDEE3CFC900002ECF030
:1060C000A3EDF090004BE0D39401401A900002E061
:1060D000FEA3E0FFAC55AD56EF2DFDEE3CFC90006D
:1060E00002ECF0A3EDF0D210AE53AF54900002E0FA
:1060F000FCA3E0FDEFC39DEE9C400D124A54D295E7
:10610000C21074C890004AF0A210B3B350079000B8
:106110004AE0B55E02800D124A54D29574C89000D0
:106120004AF0C21090004CE0B55E0280030261C3E9
:10613000A211407290000EE0FEA3E0FFEF4E60213E
:10614000AE55AF5690000EE0FCA3E0FD12000374C4
:106150000A8E048F05FF1271A290000EECF0A3EDE1
:10616000F090004DE0601A90000EE0FEA3E0FFAC5E
:1061700055AD56EF2DFDEE3CFC90000EECF0A3ED7E
:10618000F090004DE0D39401401A90000EE0FEA381
:10619000E0FFAC55AD56EF2DFDEE3CFC90000EEC53
:1061A000F0A3EDF0D211AE53AF5490000EE0FCA37B
:1061B000E0FDEFC39DEE9C400AC295744690004CF2
:1061C000F0C211A211B3B3500790004CE0B55E02CB
:1061D000800AC295744690004CF0C21190004EE0C7
:1061E000B55E02800302627EA2124072900004E05B
:1061F000FEA3E0FFEF4E6021AE55AF56900004E0E5
:10620000FCA3E0FD120003740A8E048F05FF1271D7
:10621000A2900004ECF0A3EDF090004FE0601A9023
:106220000004E0FEA3E0FFAC55AD56EF2DFDEE3CC3
:10623000FC900004ECF0A3EDF090004FE0D394014B
:10624000401A900004E0FEA3E0FFAC55AD56EF2DE0
:10625000FDEE3CFC900004ECF0A3EDF0D212AE5346
:10626000AF54900004E0FCA3E0FDEFC39DEE9C4022
:106270000D124A54D2A0C21274C890004EF0A2125D
:10628000B3B3500790004EE0B55E02800D124A5441
:10629000D2A074C890004EF0C212900050E0B55EDB
:1062A000028003026339A2134072900010E0FEA343
:1062B000E0FFEF4E6021AE55AF56900010E0FCA31A
:1062C000E0FD120003740A8E048F05FF1271A29084
:1062D0000010ECF0A3EDF0900051E0601A90001077
:1062E000E0FEA3E0FFAC55AD56EF2DFDEE3CFC907B
:1062F0000010ECF0A3EDF0900051E0D39401401AAF
:10630000900010E0FEA3E0FFAC55AD56EF2DFDEE82
:106310003CFC900010ECF0A3EDF0D213AE53AF5460
:10632000900010E0FCA3E0FDEFC39DEE9C400AC28C
:10633000A07446900050F0C213A213B3B35007905C
:106340000050E0B55E02800AC2A07446900050F092
:10635000C213900052E0B55E0280030263F4A214FF
:106360004072900006E0FEA3E0FFEF4E6021AE55C4
:10637000AF56900006E0FCA3E0FD120003740A8E05
:10638000048F05FF1271A2900006ECF0A3EDF090CF
:106390000053E0601A900006E0FEA3E0FFAC55ADAC
:1063A00056EF2DFDEE3CFC900006ECF0A3EDF090D6
:1063B0000053E0D39401401A900006E0FEA3E0FFF2
:1063C000AC55AD56EF2DFDEE3CFC900006ECF0A375
:1063D000EDF0D214AE53AF54900006E0FCA3E0FD04
:1063E000EFC39DEE9C400D124A54D297C21474C85C
:1063F000900052F0A214B3B35007900052E0B55E83
:1064000002800D124A54D29774C8900052F0C21400
:10641000900054E0B55E0280030264AFA2154072A2
:10642000900012E0FEA3E0FFEF4E6021AE55AF56A4
:10643000900012E0FCA3E0FD120003740A8E048FAA
:1064400005FF1271A2900012ECF0A3EDF090005540
:10645000E0601A900012E0FEA3E0FFAC55AD56EFED
:106460002DFDEE3CFC900012ECF0A3EDF0900055F9
:10647000E0D39401401A900012E0FEA3E0FFAC5577
:10648000AD56EF2DFDEE3CFC900012ECF0A3EDF0CC
:10649000D215AE53AF54900012E0FCA3E0FDEFC361
:1064A0009DEE9C400AC2977446900054F0C215A21B
:1064B00015B3B35007900054E0B55E02800AC2974E
:1064C0007446900054F0C215900056E0B55E02800C
:1064D0000302656AA2164072900008E0FEA3E0FF86
:1064E000EF4E6021AE55AF56900008E0FCA3E0FDF2
:1064F000120003740A8E048F05FF1271A290000827
:10650000ECF0A3EDF0900057E0601A900008E0FE78
:10651000A3E0FFAC55AD56EF2DFDEE3CFC9000081E
:10652000ECF0A3EDF0900057E0D39401401A9000F6
:1065300008E0FEA3E0FFAC55AD56EF2DFDEE3CFCB0
:10654000900008ECF0A3EDF0D216AE53AF549000DB
:1065500008E0FCA3E0FDEFC39DEE9C400D124A5401
:10656000D2A2C21674C8900056F0A216B3B3500758
:10657000900056E0B55E02800D124A54D2A274C853
:10658000900056F0C216900058E0B55E02800302FB
:106590006625A2174072900014E0FEA3E0FFEF4EC4
:1065A0006021AE55AF56900014E0FCA3E0FD120050
:1065B00003740A8E048F05FF1271A2900014ECF090
:1065C000A3EDF0900059E0601A900014E0FEA3E003
:1065D000FFAC55AD56EF2DFDEE3CFC900014ECF0F9
:1065E000A3EDF0900059E0D39401401A900014E01C
:1065F000FEA3E0FFAC55AD56EF2DFDEE3CFC900048
:1066000014ECF0A3EDF0D217AE53AF54900014E0A9
:10661000FCA3E0FDEFC39DEE9C400AC2A27446902D
:106620000058F0C217A217B3B35007900058E0B556
:106630005E02800AC2A27446900058F0C217900011
:106640005AE0B55E0280030266E0A2184072900034
:106650000AE0FEA3E0FFEF4E6021AE55AF5690007A
:106660000AE0FCA3E0FD120003740A8E048F05FF0C
:106670001271A290000AECF0A3EDF090005BE060D4
:106680001A90000AE0FEA3E0FFAC55AD56EF2DFDD9
:10669000EE3CFC90000AECF0A3EDF090005BE0D340
:1066A0009401401A90000AE0FEA3E0FFAC55AD56FD
:1066B000EF2DFDEE3CFC90000AECF0A3EDF0D218BB
:1066C000AE53AF5490000AE0FCA3E0FDEFC39DEE93
:1066D0009C400D124A54D2A1C21874C890005AF0BE
:1066E000A218B3B3500790005AE0B55E02800D12B5
:1066F0004A54D2A174C890005AF0C21890005CE0CD
:10670000B55E02800302679BA2194072900016E0FA
:10671000FEA3E0FFEF4E6021AE55AF56900016E0AD
:10672000FCA3E0FD120003740A8E048F05FF1271B2
:10673000A2900016ECF0A3EDF090005DE0601A90DE
:106740000016E0FEA3E0FFAC55AD56EF2DFDEE3C8C
:10675000FC900016ECF0A3EDF090005DE0D3940106
:10676000401A900016E0FEA3E0FFAC55AD56EF2DA9
:10677000FDEE3CFC900016ECF0A3EDF0D219AE5308
:10678000AF54900016E0FCA3E0FDEFC39DEE9C40EB
:106790000AC2A1744690005CF0C219A219B3B350AA
:1067A0000790005CE0B55E02800AC2A174469000CA
:1067B0005CF0C2199000FDE0B4020280030268DCC4
:1067C000900095E0D395665064900095E0F4042520
:1067D00066FE900100E08E00F5F0E884FF7E008FF9
:1067E00073EFC39410500CEF8573F0A4FDACF08DE3
:1067F0007380037573FF900095E0D39573400B9001
:106800000095E0C39573F571800375710090011BCD
:10681000E0D39571400690011BE0F57190011CE0FA
:10682000C39571500690011CE0F571807190009540
:10683000E0C39566FE900100E08E00F5F0E884FF6D
:106840007E008F73EFC39410500CEF8573F0A4FD9E
:10685000ACF08D7380037573FF85735A7559009082
:106860000095E0255AFFAE5950010E8E598F5A748B
:10687000FFBE0009D39F4005855A7180037571FFE3
:1068800090011BE0D39571400690011BE0F57190DB
:10689000011CE0C39571500690011CE0F571A20344
:1068A000B3B3500D900096E0FE900108E0D39E50E7
:1068B00002800E7407900075F0E5B554BFF5B58001
:1068C0001B75A710E5CDC395714008E5B554BFF51C
:1068D000B58006E5B54440F5B575A700900122E006
:1068E000A851B80005D395525016900121E0A85147
:1068F000B8000D95524009900123E0D39561400204
:10690000802975A710E5CDC394BF400EE5B554EFBF
:10691000F5B5E5B554DFF5B5800CE5B54410F5B532
:10692000E5B54420F5B575A700802775A710E5CD1E
:10693000C39440400EE5B554EFF5B5E5B554DFF529
:10694000B5800CE5B54410F5B5E5B54420F5B57551
:10695000A700E56FC39413501DE56F75F00284AF77
:10696000F07E00EF4E70051232FC800AA2EDB340BB
:1069700005C2ED1232FCAE53AF547498C39F743A03
:106980009E400C900094E0C3945A4003026AB8A25F
:1069900008B340091246F97406900075F0A20AB3D4
:1069A000500EE561D394334007E561C394CC4002B7
:1069B000804190012DE0B40214121281900098E001
:1069C00075F05EA4FFAEF08E5B8F5C800F9000A927
:1069D000E075F05EA4FFAEF08E5B8F5CE55C455B1E
:1069E0006011E5B54401F5B5741F900093F01249AC
:1069F000A2D20A900094E0D394014007E561C394C9
:106A00001A40028002C20A9006ECE0600675080196
:106A1000122E4F9006F0E06006750802122E4F907D
:106A200006F4E06006750803122E4F9006F8E06049
:106A300006750804122E4F900094E0C3945A50102B
:106A4000E56FB41309900094E004F0756F00803F87
:106A5000E56FB41303756F00C28E758D00758B00E2
:106A6000756400755401755300D28E900093E0C395
:106A7000942E5008900093E004F08006742E90004D
:106A800093F0900093E0B42E06E5B554FEF5B59072
:106A90000094E0D394014007E56AC394414002802A
:106AA00006740E900075F09008BCE0600690012A14
:0B6AB000E060028003120BD7024EC012
:106B66000000010001400160018001A001C001E0B8
:106B760002000300039603B603D603F404000500DF
:106B86000512052405360548055A056C057E05904F
:106B960005A805C005DE0600061406280646066E8C
:106BA60006AE05CF06EE00FF013F015F017F019FA4
:106BB60001BF01DF01FF02FF039503B503D503F310
:106BC60003FF04FF05110523053505470559056B28
:106BD600057D058F05A705BF05CE05F1061306271A
:106BE6000645066D06AD06ED05DD06FF0FAA0FA5E7
:106BF6000F9F0F9A0F940F8D0F870F800F780F71CD
:106C06000F680F600F570F4E0F450F3B0F300F25C4
:106C16000F1A0F0E0F020EF50EE80EDB0ECC0EBE8F
:106C26000EAE0E9F0E8E0E7D0E6C0E5A0E470E3455
:106C36000E200E0C0DF70DE20DCB0DB50D9D0D853D
:106C46000D6D0D540D3A0D200D050CE90CCE0CB151
:106C56000C940C760C580C3A0C1B0BFB0BDB0BBB89
:106C66000B9A0B790B570B350B130AF10ACE0AABAD
:106C76000A870A640A400A1C09F809D409B0098C73
:106C860009670943091F08FB08D608B2088E086A77
:106C96000846082307FF07DC07B90796077307515D
:106CA600072F070D06EC06CA06AA068906690649D5
:106CB600062A060A05EC05CD05B0059205750558A8
:106CC600053C0520050504EA04CF04B5049C0482AE
:106CD6000469045104390422040B03F403DE03C8D7
:106CE60003B2039D038903750361034D033B032828
:106CF6000316030402F202E102D102C002B002A0AE
:106D0600029102820273026502570249023C022F77
:106D160002220216020901FD01F201E601DB01D0A1
:106D260001C601BB01B101A7019D0194018B01823E
:106D36000179017001680160015801500148014163
:106D460001390132012B0125011E01180111010B28
:106D5600010500FF00FA0FA60FA00F990F920F8BE7
:106D66000F840F7C0F740F6B0F620F580F4E0F437B
:106D76000F380F2C0F1F0F120F050EF70EE80ED847
:106D86000EC80EB70EA50E930E800E6C0E580E4250
:106D96000E2C0E150DFD0DE40DCB0DB10D950D79D7
:106DA6000D5D0D3F0D200D010CE10CC00C9E0C7C01
:106DB6000C590C350C100BEA0BC40B9E0B760B4FC3
:106DC6000B260AFD0AD40AAA0A800A550A2A09FFCE
:106DD60009D409A8097C0950092508F908CD08A194
:106DE6000875084A081E07F307C8079D0773074971
:106DF600072006F706CE06A6067E06570630060AC2
:106E060005E405BF059B057705540532051004EF1B
:106E160004CE04AE048F047104530435041903FD33
:106E260003E203C703AD0394037B0363034B0334FD
:106E3600031E030802F302DE02CA02B602A302918F
:106E4600027F026D025C024C023C022C021D020E05
:106E5600020001F201E401D701CA01BE01B101A697
:106E6600019A018F0185017A01700166015D015366
:106E7600014A01410139013101290121011901129A
:106E8600010B010400FD00F700F000EA00E400DE5B
:106E960000D900D300CE00C900C400BF00BA00B5B7
:106EA60000B100AD00A800A400A0009C00990095C8
:106EB6000091008E008A008700840081007E007B9E
:10009E0075B50075840175A70075FFA075EF069004
:1000AE000071E4F075C91075A70F75A1C775A7008B
:1000BE0075D90075CE0C75A70F75F1FE75F2FF752B
:1000CE00F30775F47875A4BA75A5FF75A60775AE16
:1000DE000075AFFF75D48175D5FF75D6FF75D7FF47
:1000EE0075A70075A20175A14775F8092275E60876
:1000FE0075E71075BC0175BE0475BD6C75BE0775D0
:10010E00BDA075BE0875BD0175BC0075BB1875BC6C
:10011E002075BA0875E88075D11375A70F75E105BE
:10012E0075E20075C7401246F97597007597807491
:10013E000A1271927597C0E5975420700280F87577
:10014E008F0275A700D2AF75980075A90C75A70F11
:10015E0075AB4375ADFB75AC1E75A71075C91875DB
:10016E00CA0075CB0075C80475A700758912758E07
:10017E0004758C00758A00C2A9D28C758D00758BA2
:10018E0000D2ABD28E75B62075D944C2992290009A
:10019E00A7E09008BBF09000B2E09008BCF0900091
:1001AE00B3E09008BDF09000D2E09008BEF0900051
:1001BE00DFE09008BFF09000EDE09008C0F09000F6
:1001CE00FBE09008C1F09000FDE09008C2F09001B5
:1001DE000BE09008C3F0900118E09008C4F0900175
:1001EE0019E09008C5F090012BE09008C6F0900140
:1001FE0043E09008C8F0900191E09008C9F090019A
:10020E0092E09008CAF0900193E09008CBF0900134
:10021E002AE09008CCF0900114E09008CDF0900008
:10022E00CBE09008CEF09000CCE09008CFF090009C
:10023E00C6E09008D0F09000C7E09008D1F0900191
:10024E0030E09008D2F0900131E09008D3F09001A8
:10025E0032E09008D4F0900133E09008D5F0900190
:10026E0034E09008D6F09006EBE09008D7F09006B8
:10027E00EFE09008D8F09006F3E09008D9F09006E1
:10028E00F7E09008DAF09006FBE09008DBF09006BD
:10029E00FFE09008DCF0900703E09008DDF0900797
:1002AE0007E09008DEF090070BE09008DFF0900773
:1002BE000FE09008E0F0900793E09008E1F09007CF
:1002CE0094E09008E2F0900795E09008E3F0900734
:1002DE0096E09008E4F0900797E09008E5F090071C
:1002EE0098E09008E6F0900799E09008E7F0900704
:1002FE009AE09008E8F090079BE09008E9F09007EC
:10030E009CE09008EAF090079DE09008EBF09007D3
:10031E009EE09008ECF090079FE09008EDF09007BB
:10032E00A0E09008EEF09007A1E09008EFF09007A3
:10033E00A2E09008F0F09007A3E09008F1F0900191
:10034E0035E09008F2F0900136E09008F3F090015D
:10035E0037E09008F4F0900138E09008F5F0900145
:10036E0039E09008F6F090013AE09008F7F090012D
:10037E003BE09008F8F090013CE09008F9F0900115
:10038E003DE09008FAF090013EE09008FBF09000FE
:10039E00D9E09008FCF0900111E09008FDF090017A
:1003AE0049E09008FEF090014AE09008FFF022909C
:1003BE0008BBE09000A7F09008BCE09000B2F0906F
:1003CE0008BDE09000B3F09008BEE09000D2F0902F
:1003DE0008BFE09000DFF09008C0E09000EDF090D4
:1003EE0008C1E09000FBF09008C2E09000FDF09094
:1003FE0008C3E090010BF09008C4E0900118F09053
:10040E0008C5E0900119F09008C6E090012BF0901D
:10041E0008C8E0900143F09008CCE090012AF090DB
:10042E0008CDE0900114F09008CEE09000CBF09053
:10043E0008CFE09000CCF09008D0E09000C6F0908D
:10044E0008D1E09000C7F09008D2E0900130F09013
:10045E0008D3E0900131F09008D4E0900132F09092
:10046E0008D5E0900133F09008D6E0900134F0907A
:10047E0008D7E09006EBF09008D8E09006EFF090E9
:10048E0008D9E09006F3F09008DAE09006F7F090C5
:10049E0008DBE09006FBF09008DCE09006FFF090A1
:1004AE0008DDE0900703F09008DEE0900707F0907B
:1004BE0008DFE090070BF09008E0E090070FF09057
:1004CE0008E1E0900793F09008E2E0900794F09036
:1004DE0008E3E0900795F09008E4E0900796F0901E
:1004EE0008E5E0900797F09008E6E0900798F09006
:1004FE0008E7E0900799F09008E8E090079AF090EE
:10050E0008E9E090079BF09008EAE090079CF090D5
:10051E0008EBE090079DF09008ECE090079EF090BD
:10052E0008EDE090079FF09008EEE09007A0F090A5
:10053E0008EFE09007A1F09008F0E09007A2F0908D
:10054E0008F1E09007A3F09008F2E0900135F090EA
:10055E0008F3E0900136F09008F4E0900137F09047
:10056E0008F5E0900138F09008F6E0900139F0902F
:10057E0008F7E090013AF09008F8E090013BF09017
:10058E0008F9E090013CF09008FAE090013DF090FF
:10059E0008FBE090013EF09008FCE09000D9F0904E
:1005AE0008FDE0900111F09008FEE0900149F090F6
:1005BE0008FFE090014AF0227547009008B3E4F07E
:1005CE00A3F0753100753000754D00754E00C227D1
:1005DE00D2289008BCE06002D22074FE9008B5F8D4
:1005EE00E4F0E8A3F074FE9008B9F8E4F0E8A3F0A4
:1005FE0074FE9008B7F8E4F0E8A3F0745A90090D71
:10060E00F0745A90090EF0D229C225C22BC22AC20A
:10061E0026C22DC23322750B00750A00AE0AAF0B2F
:10062E00AC08AD09EDC39FEC9E401674FF1271929B
:10063E0075CF01780B740126F6500418E436F65087
:10064E00DB22C2AF75D904758F0375B7A575B7F1E7
:10065E0090F800E4F0758F0175B7A575B7F1E52731
:10066E0090F800F075B7A575B7F190F801E4F07544
:10067E00B7A575B7F1900901E090F802F075B7A52E
:10068E0075B7F1900905E090F803F075B7A575B749
:10069E00F1900902E090F804F075B7A575B7F190E6
:1006AE000903E090F805F075B7A575B7F190090448
:1006BE00E090F806F075B7A575B7F1900906E090D1
:1006CE00F807F0758F0075D944D2AF22900071E013
:1006DE00B4AB61C2AF75D90475B62275F522758FAC
:1006EE000375B7A575B7F1740090F600F0758F011C
:1006FE00755A00755900AE59AF5A7445BE00279F02
:10070E00402475B7A575B7F19008BB120048E0FC00
:10071E0090F600120048ECF0785A740126F6500458
:10072E0018E436F650D0758F0075F51175B6207534
:10073E00D944D2AF22C2AF75F52275D904755A00CD
:10074E00755900AE59AF5A7445BE00229F401F9096
:10075E00F600120048E493FC9008BB120048ECF03F
:10076E00785A740126F6500418E436F650D575D929
:10077E004475F511D2AF22900071E0B4AA02800345
:10078E000208C2C2AF75D90475B62275F522758FEF
:10079E000375B7A575B7F1740090F400F075B7A5A1
:1007AE0075B7F1740090F200F075B7A575B7F174D6
:1007BE000090F000F075B7A575B7F1740090EE00DB
:1007CE00F0758F01755A00755900AE59AF5A74FF06
:1007DE00C39F74019E402475B7A575B7F19000A50F
:1007EE00120048E0FC90F400120048ECF0785A74C5
:1007FE000126F6500418E436F650CF755A00755996
:10080E0000AE59AF5A74FFC39F74019E402475B752
:10081E00A575B7F19002A5120048E0FC90F2001207
:10082E000048ECF0785A740126F6500418E436F6B7
:10083E0050CF755A00755900AE59AF5A74FFC39F09
:10084E0074019E402475B7A575B7F19004A51200EA
:10085E0048E0FC90F000120048ECF0785A74012643
:10086E00F6500418E436F650CF755A00755900AE9E
:10087E0059AF5A74FFC39F74019E402475B7A57576
:10088E00B7F19006A5120048E0FC90EE0012004869
:10089E00ECF0785A740126F6500418E436F650CF70
:1008AE00758F0075F51175B62075D944D2AF743AAF
:1008BE009007A5F022900071E0B4AA028003020A0C
:1008CE0000C2AF75D90475B62275F522758F037502
:1008DE00B7A575B7F1740090EC00F075B7A575B7B4
:1008EE00F1740090EA00F075B7A575B7F174009039
:1008FE00E800F075B7A575B7F1740090E600F075D5
:10090E008F01755A00755900AE59AF5A74FFC39FC7
:10091E0074019E402475B7A575B7F19000A512001D
:10092E0048E0FC90EC00120048ECF0785A74012676
:10093E00F6500418E436F650CF755A00755900AECD
:10094E0059AF5A74FFC39F74019E402475B7A575A5
:10095E00B7F19002A5120048E0FC90EA00120048A0
:10096E00ECF0785A740126F6500418E436F650CF9F
:10097E00755A00755900AE59AF5A74FFC39F740172
:10098E009E402475B7A575B7F19004A5120048E0F6
:10099E00FC90E800120048ECF0785A740126F650EC
:1009AE000418E436F650CF755A00755900AE59AF9B
:1009BE005A74FFC39F74019E402475B7A575B7F195
:1009CE009006A5120048E0FC90E600120048ECF0FC
:1009DE00785A740126F6500418E436F650CF758F07
:1009EE000075F51175B62075D944D2AF743A9007DB
:1009FE00A5F022C2AF75D90475F522755A00755946
:100A0E0000AE59AF5A74FFC39F74019E401F90F4FD
:100A1E0000120048E493FC9000A5120048ECF07818
:100A2E005A740126F6500418E436F650D4755A005E
:100A3E00755900AE59AF5A74FFC39F74019E401F83
:100A4E0090F200120048E493FC9002A5120048ECCC
:100A5E00F0785A740126F6500418E436F650D47520
:100A6E005A00755900AE59AF5A74FFC39F74019E58
:100A7E00401F90F000120048E493FC9004A5120071
:100A8E0048ECF0785A740126F6500418E436F65005
:100A9E00D4755A00755900AE59AF5A74FFC39F747E
:100AAE00019E401F90EE00120048E493FC9006A5B4
:100ABE00120048ECF0785A740126F6500418E43609
:100ACE00F650D475F51175D944D2AF74019000EE7D
:100ADE00F0743A9007A5F09009147401F022C2AF99
:100AEE0075D90475F522755A00755900AE59AF5A6D
:100AFE0074FFC39F74019E401F90EC00120048E4E7
:100B0E0093FC9000A5120048ECF0785A740126F67A
:100B1E00500418E436F650D4755A00755900AE5983
:100B2E00AF5A74FFC39F74019E401F90EA001200DB
:100B3E0048E493FC9002A5120048ECF0785A740138
:100B4E0026F6500418E436F650D4755A007559003E
:100B5E00AE59AF5A74FFC39F74019E401F90E800B8
:100B6E00120048E493FC9004A5120048ECF0785A69
:100B7E00740126F6500418E436F650D4755A0075F2
:100B8E005900AE59AF5A74FFC39F74019E401F9017
:100B9E00E600120048E493FC9006A5120048ECF023
:100BAE00785A740126F6500418E436F650D475F5CA
:100BBE001175D944D2AF74029000EEF0743A9007DA
:100BCE00A5F07402900914F02274019000EEF090DA
:100BDE0008BCE0903CBBF828287380188016A2A3AE
:100BEE00400674029000EEF0800AA2A44006740241
:040BFE009000EEF085
:0C3CBB00020BE8020BEA020BEC020BF813
:100C02009000EEE0B40105A231B34002801AD23165
:100C12001246F9120A0174019000EEF01203BD129D
:100C22003E57741B900075F09000EEE0B40206A2ED
:100C320031B3B34002801AC2311246F9120AEC747F
:100C4200029000EEF01203BD123E57741B90007525
:100C5200F022E54E64046006E59964FF600280318B
:100C6200A2274004D2278027E54E600874E6254E6D
:100C7200900075F0E54D600874F0254D900075F018
:100C8200E54EB4010280FE754E00754D00C227800C
:100C920002C227E54E903CC7F8282873754E00E53E
:100CA20099B4FF03754D01E599B4FE03754D02E554
:100CB20099B4FD03754D03E599B4FC03754D04E544
:100CC20099B4FA03754D05E599B4FB06754E011208
:100CD20046F9E599B4F906754E041246F9E599B458
:100CE200F7331246F9C29C74AB900071F01206DA27
:100CF20074AA900071F0900914E0B40105120785FE
:100D020080031208C3900071E4F0D29C754E007506
:100D12004D007599F7E599D394E54007E599C39499
:100D2200F04002801685994F754E027E017F00E5E4
:100D32004FC394E61271B28E328F339008B3E4F04F
:100D4200A3F0E599D394C24007E599C394E6400223
:100D5200802885994F754E0374E5C3954FF5337519
:100D62003200AE32AF33906B66127181E493F87445
:100D720001939008B3C8F0A3C8F0D2990210DF9093
:100D820008C8E0700AA221B35005A222B340028033
:100D92005C9008B3E0FEA3E0FF74FFBE00039F5027
:100DA20009EFC39446EE9406402B9008B3E0FEA3ED
:100DB200E0FFEFD3946DEE94064009EFC394EEEE9C
:100DC200940640119008B3E0FEA3E0FFEFD394FF36
:100DD200EE940640139008B3E0FEA3E0FF9000A556
:100DE200120048E599F0800385997480119008B348
:100DF200E0FEA3E0FF9000A5120048E599F09008FC
:100E0200B31271C09008B3E0FEA3E0FFEFB4010695
:100E1200EEB407028003020EDA9007A5E0B43C02AA
:100E22008003020EDAA221B35005A222B34002804F
:100E320055C29C1203BD9000B2E0900913F0123F1C
:100E420092900191E09008C9F0900192E09008CA56
:100E5200F0900193E09008CBF074AB900071F01227
:100E620006DA74AA900071F0900914E0B401051238
:100E7200078580031208C3900914E09000EEF090F9
:100E82000071E4F08047C29C12019C74009008C972
:100E9200F074009008CAF074009008CBF09000B291
:100EA200E0900913F0123F9274AB900071F01206B9
:100EB200DA74AA900071F01207851208C3D29C75E9
:100EC20099FB75096475080012062480FED29C7590
:100ED2004E00754D007599FB0210DF9008B3E0FEDD
:100EE200A3E0FFEF4E70068599317530009008B38C
:100EF200E0FEA3E0FF74016F4E701BAC30AD31AA6F
:100F020032AB33ED2BFBEC3AFA8A068B079000A545
:100F1200120048E599F09008B31271C09008B3E04E
:100F2200FEA3E0FF74026F4E7021AC30AD317456F7
:100F32006D4C7006E54F64E6600280031246F912BA
:100F42003F92854F99754E00754D000210DF900853
:100F5200B3E0FEA3E0FF9000A5120048E599F090EF
:100F620008B31271C09008B3E0FEA3E0FFAC32AD4B
:100F7200338F028E038C068D07906BAC127181E465
:100F820093F9740193FEEAD39EEB994009854F9938
:100F9200754E00754D000210DF9008B3E0FEA3E02D
:100FA200FF9000A5120048E599F09008B31271C0B5
:100FB2009008B3E0FEA3E0FFEFB40006EEB4010236
:100FC20080030210DF900087E0D394C7400B9000AB
:100FD20087E0C394C8F550801A900087E0D39463E9
:100FE200400B900087E0C39464F550800690008720
:100FF200E0F550E55075F002A4FFAEF08F73EF906C
:1010020000A51271E3EFFCE0FDEC9000A81271E381
:10101200EDFCE0FDEC2DB5500280030210D10FEF84
:101022009000A51271E3E573FFE0FCEF9000A912B6
:1010320071E3ECFFE0FCEFC39CB5500280030210A9
:10104200D1E5739000A71271E3E573FFE0FCEF9026
:1010520000AA1271E3ECFFE0FCEF2CB55071E573CE
:101062009000AB1271E3E0C39550900901F0E57373
:101072009000AC1271E3E0C39550900902F0E57361
:101082009000AF1271E3E0C39550900903F0E5734D
:101092009000B01271E3E0C39550900904F0E5733B
:1010A2009000B11271E3E0C39550900905F0E57329
:1010B2009000B21271E3E0C39550900906F0120657
:1010C200507599F975096475080012062480FE7539
:0D10D20099FF75096475080012062480FE60
:0F3CC700020C9E020D81020EDD020F50020F9BB8
:1010DF0022E54D903CD6F82828730211C49008B32E
:1010EF00E0FEA3E0FF900077120048E0F59990082A
:1010FF00B31271C09008B3E0FEA3E0FF741C6F4EF3
:10110F007003754D000211C4856E990211C49008C9
:10111F00B3E0FEA3E0FF9000A5120048E0F599EFC1
:10112F00B40107EEB40703754D009008B31271C0F8
:07113F000211C49008B4E0A6
:0F3CD6000210E90210EC02111702111D02114237
:10114600903D48F82828738552998067855F998075
:1011560062856199805D8565998058856799805318
:10116600856899804E8569998049856A99804490F9
:101176000027E0F599803CA228B340077599FAC28A
:10118600288017A220B3400575990F800B90007533
:10119600E0F599900075E4F0C2208017856B998080
:1011A60012856699800D856C9980087599FC800377
:0311B600754D0074
:103D480002114D02115202115702115C0211610257
:103D5800116602116B02117002117502117D0211B8
:0D3D6800A20211A70211AC0211B10211B6A6
:0B11B9009008B31271C08003123EB218
:033CE5000211C108
:1011C40022E537255AFFAE5950010E9000A51200B2
:1011D40048E0F538E537255AFFAE5950010E0FBFE8
:1011E40000010E9000A5120048E0F539853F3BE56B
:1011F40038B539058538378041E539D39538401DF0
:10120400E539C39538853AF0A4FFAEF0E53B8E048A
:101214008F05FF1271A2ED2538F537801DE538C31F
:101224009539853AF0A4FFAEF0E53B8E048F05FFB7
:101234001271A2EDF4042538F53722E539D3953837
:10124400401DE539C39538853AF0A4FFAEF0E53B7F
:101254008E048F05FF1271A2ED2538F537801DE548
:1012640038C39539853AF0A4FFAEF0E53B8E048F80
:1012740005FF1271A2EDF4042538F537229000AB76
:10128400E0B4017FE56775F00A84FF7E008F37E5DF
:101294006775F00A84ADF07C008D3A753F0A755984
:1012A40005755A24E537C3941150051211C58006FB
:1012B4009005DAE0F537E537C394F05008E5379048
:1012C4000098F0800674EF900098F0E56775F00AD6
:1012D40084FF7E008F37E56775F00A84ADF07C00EB
:1012E4008D3A753F0A755905755A5AE537C39411F5
:1012F40050051211C58006900610E0F537E53790C9
:101304000070F0229000ABE0B40102800302139657
:10131400E56775F00A84FF7E008F37E56775F00A8C
:1013240084ADF07C008D3A753F0A755905755A36BF
:10133400E537C3941150051211C580069005ECE001
:10134400F537E537C394F0500585374B8003754B6B
:10135400EFE56775F00A84FF7E008F37E56775F067
:101364000A84ADF07C008D3A753F0A755905755AAB
:1013740048E537C3941150051211C580069005FE47
:10138400E0F537E537C394F0500585374C80037595
:101394004CEF22E55F75F00484FF7E008F37E55F34
:1013A40075F00484ADF07C008D3A753F04755901E5
:1013B400755A00E537C3943F50051211C580069055
:1013C40001E4E0F537E5379008ADF8E4F0E8A3F080
:1013D400900074E075F020A4FFAEF09000F6E08E6B
:1013E400048F05FF1271A28D379000DEE0D3955F64
:1013F40050030214A2900102E0D3955F4010ED90D7
:1014040001E51271E3E0F52B752A0002149F9000A8
:10141400CDE0D3955F4043E5379001E51271E3E0F9
:10142400F538E5379002051271E3E0F539900102D1
:10143400E0F404255FF53A9000CDE0FE900102E06F
:10144400F4042EF53BE538B53905853837800312A9
:10145400123F85372B752A008041E537900205122B
:1014640071E3E0F538E5379002251271E3E0F539D0
:101474009000CDE0F404255FF53A9000DEE0FE90A4
:1014840000CDE0F4042EF53BE538B5390585383751
:10149400800312123F85372B752A000215499001EB
:1014A40005E0D3955F5011E5379002651271E3E0D2
:1014B400F52B752A000215499000CEE0D3955F50B4
:1014C40043E5379002451271E3E0F538E5379002C1
:1014D400651271E3E0F5399000CEE0F404255FF580
:1014E4003A900105E0FE9000CEE0F4042EF53BE5D1
:1014F40038B53905853837800312123F85372B7587
:101504002A008041E5379002251271E3E0F538E5C1
:10151400379002451271E3E0F5399000DEE0F404FF
:10152400255FF53A9000CEE0FE9000DEE0F4042E54
:10153400F53BE538B53905853837800312123F8508
:10154400372B752A0022900116E0F53C753F117582
:101554005902755A00AE51AF52E53C75F00FA4FD27
:10156400ACF0EDD39FEC9E4021E53C8E048F05FF4B
:101574001271A2ED75F010A4FFAEF0E55F75F011E5
:1015840084FD7C00ED2FF53D800EE55F75F0118440
:10159400FF7E00EF24F0F53D853D37E55F75F011E2
:1015A40084AFF07E008F3A1211C585373EAE51AF3D
:1015B40052900116E075F00FA4FDACF0EDD39FEC52
:1015C4009E4028755902755A10853D371211C585FC
:1015D4003E38853739AE51AF52E53C8E048F05FF56
:1015E4001271CD8D3A853C3B12123FE5379008AD20
:1015F400F8E4F0E8A3F0752B64752A002290011634
:10160400E0F53C753F11755902755A00AE51AF5261
:10161400E53C75F00FA4FDACF0EDD39FEC9E4021AA
:10162400E53C8E048F05FF1271A2ED75F010A4FF46
:10163400AEF0E56175F01184FD7C00ED2FF53D8081
:101644000EE56175F01184FF7E00EF24F0F53D8511
:101654003D37E56175F01184AFF07E008F3A1211C9
:10166400C585373EAE51AF52900116E075F00FA418
:10167400FDACF0EDD39FEC9E4028755902755A10CD
:10168400853D371211C5853E38853739AE51AF5285
:10169400E53C8E048F05FF1271CD8D3A853C3B12DB
:1016A400123FE5379008ADF8E4F0E8A3F0E56B608D
:1016B40017E56BC394FE501090010AE0B402099040
:1016C40000F8E0D3940B5002801F9008ADE0FEA315
:1016D400E0FFE56B1271B274E78E048F05FF12719F
:1016E400A29008ADECF0A3EDF09000E0E0B4045F4C
:1016F400E55F75F00484FF7E008F37E55F75F004C5
:1017040084ADF07C008D3A753F04755901755A001B
:10171400E537C3943F50051211C580069001E4E0FB
:10172400F5379008ADE0FEA3E0FFE5371271B2741F
:10173400328E048F05FF1271A29008ADE0FEA3E083
:10174400FFEF2DFDEE3CFC9008ADECF0A3EDF07541
:101754002B64752A00229000ABE0B40146E567755E
:10176400F00A84FF7E008F37E56775F00A84ADF0D8
:101774007C008D3A753F0A755905755A00E537C3E3
:10178400941150051211C580069005B6E0F537AEE8
:101794002AAF2BE5372FFF50010E74641271F58EBA
:1017A4002A8F2B9000ACE0B40146E56875F00A84FA
:1017B400FF7E008F37E56875F00A84ADF07C008DFC
:1017C4003A753F0A755905755A6CE537C39411503B
:1017D400051211C58006900622E0F537AE2AAF2B1C
:1017E400E5372FFF50010E74641271F58E2A8F2B8A
:1017F4009000BBE0B40249E56AC3944175F00584E6
:10180400FF7E008F37E56A75F00584ADF07C008DAE
:101814003A753F05755906755A00E537C394135058
:10182400051211C580069006B8E0F537AE2AAF2B35
:10183400E5372FFF50010E74641271F58E2A8F2B39
:101844009000FDE0B4020280030218F9E55F75F030
:101854001584FF7E008F37E55F75F01584ADF07C4D
:10186400008D3A753F15755903755AF4E537C394DD
:101874000B50051211C580069004A4E0F537E53736
:1018840075F0FFA4FFAEF09000FEE08E048F05FF1C
:101894001271A2ED900095F0E56675F078A4FFAEA4
:1018A400F074FF8E048F05FF1271A28C598D5A7447
:1018B400028C068D071200398F37AC59AD5A740467
:1018C400FF1271CD8D3A753F04755906755A28E596
:1018D40037C3941D50051211C580069006EAE0F541
:1018E40037AE2AAF2BE5372FFF50010E7464127107
:1018F400F58E2A8F2B9000AAE0B4025DE56175F0A5
:1019040064A4FFAEF074081200398E5B8F5C74051A
:101914008E048F05FF1271A28D37AE5BAF5C740528
:101924008E048F05FF1271CD8D3A753F05755905EB
:10193400755ADEE537C3941350051211C58006901D
:101944000696E0F537AE2AAF2BE5372FFF50010E90
:1019540074641271F58E2A8F2B9000ECE0707F90E6
:101964000074E075F00A84FF7E008F37900074E005
:1019740075F00A84ADF07C008D3A753F0A755905FF
:10198400755AC0E537C3940E50051211C5800690F0
:101994000673E0F537E537900099F090010BE0B459
:1019A400023C900074E075F00A84FF7E008F37904B
:1019B4000074E075F00A84ADF07C008D3A753F0A3E
:1019C400755905755ACFE537C3940E50051211C5E4
:1019D4008006900682E0F537E53790009AF0229071
:1019E40000B3E0B40117900908E0252BFFAE2A509C
:1019F400010E900107E01271F58E2A8F2B90012BB6
:101A0400E0B4011490012CE0A851B80004955250A0
:101A140007E55FC39560400280139000D5E0252B55
:101A2400FFAE2A50010E8E2A8F2B021E4A9000B35D
:101A3400E0B40306A225B3B340028050900912E03B
:101A4400701090090BE0C39405A851B80006955294
:101A5400400280109000D5E0252BFFAE2A50010EE5
:101A64008E2A8F2B900912E0600D90090BE0A8518B
:101A7400B800069552400280109000D5E0252BFF57
:101A8400AE2A50010E8E2A8F2B021E4A9000ADE022
:101A9400B402028003021E4A9000B0E0602FE567A2
:101AA400D39446402890001EE0FEA3E0FF9000EB94
:101AB400E075F003A4FDACF0EFD39DEE9C400E90D6
:101AC400010FE0A851B80005D395525003021E4AF5
:101AD4009000E0E0B403028003021C9285615A7511
:101AE40059009000B7E0A851B800049552500E90E8
:101AF40000B8E0A859B80005D3955A5003021C8FCA
:101B0400E56175F002A4FFAEF074158E048F05FF35
:101B14001271A28C068D07900635120048FEE0FF74
:101B2400EE9000AFE0FEEF8E0088F0A4FFAEF074FC
:101B3400648E048F05FF1271A28C598D5A90007423
:101B4400E075F018A4FFAEF09000F6E08E048F0567
:101B5400FF1271A28C068D0790064D120048AE59F3
:101B6400AF5AE01271B274648E048F05FF1271A231
:101B74008C598D5AE565A859B80005D3955A500378
:101B8400021C06E565C3955AFFE49559FE8E598FEC
:101B94005A7428BE00039F500C755A287559007456
:101BA4000D900075F0AE59AF5A9000B0E01271B2CA
:101BB40074288E048F05FF1271A28C598D5A9008D7
:101BC400ADE0FEA3E0FF740A8E048F05FF1271A23C
:101BD4008D068C07AC59AD5ACFCECF120003740AD0
:101BE4008E048F05FF1271A28C598D5A9008ADE0B6
:101BF400FEA3E0FF1271FD9008ADEEF0A3EFF0023A
:101C04001C8FE565A859B80004955A507EAE59AFAB
:101C14005AE5651271F58E598F5A7428BE00039FD8
:101C2400500C755A28755900740D900075F0AE5912
:101C3400AF5A9000B0E01271B274288E048F05FF81
:101C44001271A28C598D5A9008ADE0FEA3E0FF7486
:101C54000A8E048F05FF1271A28D068C07AC59AD54
:101C64005ACFCECF120003740A8E048F05FF12716F
:101C7400A28C598D5A9008ADE0FEA3E0FFEF2DFD34
:101C8400EE3CFC9008ADECF0A3EDF0021E4A90008F
:101C9400F8E0855FF0A4FFAEF074051271B274072A
:101CA4001200398E598F5A9000B7E0A851B8000439
:101CB400955250129000B8E075F002A4FDACF0EF1C
:101CC400C39DEE9C4003021E4AE55F75F00B84FF42
:101CD4007E00900635120048FEE0FFEE9000AFE073
:101CE400FEEF8E0088F0A4FFAEF074648E048F05BE
:101CF400FF1271A28C598D5A900074E075F018A4EB
:101D0400FFAEF09000F6E08E048F05FF1271A28CF6
:101D1400068D0790064D120048AE59AF5AE0127175
:101D2400B274648E048F05FF1271A28C598D5AE52A
:101D340065A859B80005D3955A5003021DC1E5653D
:101D4400C3955AFFE49559FE8E598F5A7428BE00E4
:101D5400039F500C755A28755900740D900075F046
:101D6400AE59AF5A9000B0E01271B274288E048F4D
:101D740005FF1271A28C598D5A9008ADE0FEA3E0C4
:101D8400FF740A8E048F05FF1271A28D068C07ACB6
:101D940059AD5ACFCECF120003740A8E048F05FFBB
:101DA4001271A28C598D5A9008ADE0FEA3E0FF1287
:101DB40071FD9008ADEEF0A3EFF0021E4AE565A8B0
:101DC40059B80004955A507EAE59AF5AE565127160
:101DD400F58E598F5A7428BE00039F500C755A28EB
:101DE400755900740D900075F0AE59AF5A9000B05B
:101DF400E01271B274288E048F05FF1271A28C59FF
:101E04008D5A9008ADE0FEA3E0FF740A8E048F059E
:101E1400FF1271A28D068C07AC59AD5ACFCECF12EA
:101E24000003740A8E048F05FF1271A28C598D5A17
:101E34009008ADE0FEA3E0FFEF2DFDEE3CFC900822
:101E4400ADECF0A3EDF02290010BE0B4027BE55F72
:101E540075F00884FF7E008F37E55F75F00884AD68
:101E6400F07C008D3A753F08755901755AE0E537E5
:101E7400C3943F50051211C580069002A4E0F537C3
:101E8400E5379008AFF8E4F0E8A3F09008AFE0FE7F
:101E9400A3E0FFAC2AAD2B12000374648E048F05FB
:101EA400FF1271A29008AFECF0A3EDF09000A8E04F
:101EB4008C068D071271B274648E048F05FF127143
:101EC400A29008AFECF0A3EDF09008ADE0FEA3E023
:101ED400FFAC2AAD2B12000374648E048F05FF122D
:101EE40071A29008ADECF0A3EDF09000A8E08C0690
:101EF4008D071271B274648E048F05FF1271A29063
:101F040008ADECF0A3EDF0A203401DAE51AF527446
:101F140005BE00039F5002D203E561D394CC400870
:101F2400D2017411900075F02290010AE0B4020805
:101F34009000F8E0640B600280459008ADE0FEA3D9
:101F4400E0FFE56B1271B274E78E048F05FF127126
:101F5400A29008ADECF0A3EDF090010BE0B4021FE9
:101F64009008AFE0FEA3E0FFE56B1271B274E78E58
:101F7400048F05FF1271A29008AFECF0A3EDF0906E
:101F840000CAE05402601B9000C1E0A851B80012DE
:101F9400D39552400DA203B3B35007E561C3949A9D
:101FA4004002805FAE34AF359000BFE075F002A40C
:101FB400FDACF0EF2DFDEE3CFC74022DFD50010C48
:101FC400E561BC003ED39D403A754301A22C4033E9
:101FD4009000C0E075F05EA4FDACF07405FF1271D2
:101FE400A28C5B8D5C1249A29008ADE0FEA3E0FFD9
:101FF4009000C0E02FFF50010E9008ADEEF0A3EF6B
:10200400F0D22CE561A834B8000495355002C22CF6
:10201400856135753400E543700302212390011D69
:10202400E0C39543500302211590012DE0C39402AF
:1020340040030220BFE56775F00A84FF7E00900527
:10204400A5120048E0F55A755900AE59AF5A9000F0
:10205400C0E01271B274648E048F05FF1271A28CF9
:102064005B8D5C90011DE004C395438C068D0712C3
:1020740071B290011DE08E048F05FF1271A28C5B7A
:102084008D5C9008ADE0FEA3E0FFEF2DFDEE3CFC7F
:102094009008ADECF0A3EDF090010BE0B4021A90BF
:1020A40008AFE0FEA3E0FFAA5BAB5CEF2BFBEE3ACC
:1020B400FA9008AFEAF0A3EBF0805690011DE0041B
:1020C400C39543854BF0A4FFAEF090011DE08E0450
:1020D4008F05FF1271A28C5B8D5C9008ADE0FEA3AE
:1020E400E0FFEF2DFDEE3CFC9008ADECF0A3EDF02D
:1020F40090010BE0B4021A9008AFE0FEA3E0FFAA3F
:102104005BAB5CEF2BFBEE3AFA9008AFEAF0A3EB83
:10211400F0054390011DE0C39543500375430090BF
:1021240000CAE05401601B9000BEE0A851B8001240
:10213400D39552400DA203B3B35007E55FC394CCCB
:10214400400280609000BCE075F003A4FFAEF0E5AF
:10215400402FFF50010E74032FFF50010EE55FBEA8
:102164000042D39F403E754401A22C40379000BDED
:10217400E075F05EA4FFAEF074058E048F05FF12C7
:1021840071A28C5B8D5C1249A29008ADE0FEA3E0C5
:10219400FF9000BDE02FFF50010E9008ADEEF0A3BC
:1021A400EFF0D22CE55FC395405002C22C855F400E
:1021B400E54470030222BD90011EE0C39544500320
:1021C4000222AF90012DE0C394024003022259E59C
:1021D4006775F00A84FF7E009005A5120048E0F5BB
:1021E4005A755900AE59AF5A9000BDE01271B274DD
:1021F400648E048F05FF1271A28C5B8D5C90011EAE
:10220400E004C395448C068D071271B290011EE060
:102214008E048F05FF1271A28C5B8D5C9008ADE07B
:10222400FEA3E0FFEF2DFDEE3CFC9008ADECF0A327
:10223400EDF090010BE0B4021A9008AFE0FEA3E0C9
:10224400FFAA5BAB5CEF2BFBEE3AFA9008AFEAF027
:10225400A3EBF0805690011EE004C39544854CF036
:10226400A4FFAEF090011EE08E048F05FF1271A250
:102274008C5B8D5C9008ADE0FEA3E0FFEF2DFDEEDE
:102284003CFC9008ADECF0A3EDF090010BE0B4023F
:102294001A9008AFE0FEA3E0FFAA5BAB5CEF2BFB58
:1022A400EE3AFA9008AFEAF0A3EBF0054490011E71
:1022B400E0C3954450037544009008ADE0FEA3E0EC
:1022C400FF9000CFE0BE00039F500D9000CFE09040
:1022D40008ADF8E4F0E8A3F090010BE0B40212902A
:1022E40008AFE0FEA3E0FF9000CFE0BE00059F40F2
:1022F40002800D9000CFE09008AFF8E4F0E8A3F07E
:102304002290010BE0B401028003022453A203B320
:10231400500302243A9000D6E0B4017A9008ADE06C
:10232400FEA3E0FFAC51AD52120003743C8E048F47
:1023340005FF1271A29000E6E0BC00159D401290CA
:1023440008ADE0FEA3E0FF9000E8E0BE00039F506C
:1023540002D2029008ADE0FEA3E0FFAC51AD5212F0
:102364000003743C8E048F05FF1271A29000E6E016
:10237400C3940ABC001AD39D40169008ADE0FEA396
:10238400E0FF9000E8E0C39405BE0004D39F500230
:102394008002C202807A9008ADE0FEA3E0FFAC5157
:1023A400AD5212000374788E048F05FF1271A2904F
:1023B40000E6E0BC00159D40129008ADE0FEA3E0ED
:1023C400FF9000E8E0BE00039F5004D202804190D9
:1023D40008ADE0FEA3E0FFAC51AD521200037478E7
:1023E4008E048F05FF1271A29000E6E0C3940ABC2C
:1023F400001AD39D40169008ADE0FEA3E0FF9000C4
:10240400E8E0C39405BE0004D39F50028002C202D8
:10241400A202B340219008ADE0FEA3E0FF9000E7E4
:10242400E01271B274648E048F05FF1271A29008D9
:10243400ADECF0A3EDF0A202B3400CA23040067460
:1024440024900075F0D230A2024002C2308002C251
:1024540002900070E06006A203B3B34002801990BA
:1024640008ADE0FEA3E0FF900070E02FFF50010EE6
:102474009008ADEEF0A3EFF0A200B34006A201B3C2
:10248400B35009900026E4F0A3F0802D9008ADE04D
:10249400FEA3E0FF7400D39F74019E40119008AD29
:1024A400E0F8A3E0900026C8F0A3C8F0800B74FF06
:1024B400900026F8E4F0E8A3F09000EDE0C3940463
:1024C400400C90090FE0C3940240030225AD900034
:1024D400D6E0B401479008ADE0FEA3E0FF745E12BD
:1024E40071B274058E048F05FF1271A29008ADECD1
:1024F400F0A3EDF090010BE0B4021F9008AFE0FEF2
:10250400A3E0FF745E1271B274058E048F05FF128E
:1025140071A29008AFECF0A3EDF080459008ADE017
:10252400FEA3E0FF745E1271B2740A8E048F05FF7D
:102534001271A29008ADECF0A3EDF090010BE0B4A1
:10254400021F9008AFE0FEA3E0FF745E1271B27444
:102554000A8E048F05FF1271A29008AFECF0A3ED70
:10256400F09008ADE0FEA3E0FF7402BE000CD39F20
:102574004008752902752800800A9008ADE0F52806
:10258400A3E0F5299008AFE0FEA3E0FF7402BE00CB
:102594000CD39F4008752D02752C00800A9008AF5B
:1025A400E0F52CA3E0F52D80469008ADE0FEA3E015
:1025B400FF7401BE000CD39F4008752901752800E3
:1025C400800A9008ADE0F528A3E0F5299008AFE073
:1025D400FEA3E0FF7401BE000CD39F4008752D01DB
:1025E400752C00800A9008AFE0F52CA3E0F52D903F
:1025F4000024E528F0A3E529F0A233B34009C20082
:10260400900026E4F0A3F022900074E09003A51259
:1026140071E3E0F541754264900074E0FE9000E1DE
:10262400E0D39E4037E55F75F00884FF7E008F3766
:10263400E55F75F00884ADF07C008D3A753F087550
:102644005903755A96E537C3941F50051211C58076
:102654000690045AE0F5378537428035E55F75F01A
:102664000884FF7E008F37E55F75F00884ADF07C49
:10267400008D3A753F08755903755AB6E537C3940A
:102684001F50051211C5800690047AE0F53785378E
:102694004222900117E0F53C753F11755904755AB3
:1026A40000AE51AF52E53C75F00FA4FDACF0EDD394
:1026B4009FEC9E4021E53C8E048F05FF1271A2ED34
:1026C40075F010A4FFAEF0E55F75F01184FD7C0099
:1026D400ED2FF53D800EE55F75F01184FF7E00EF70
:1026E40024F0F53D853D37E55F75F01184AFF07E4C
:1026F400008F3A1211C585373EAE51AF5290011783
:10270400E075F00FA4FDACF0EDD39FEC9E4028756E
:102714005904755A10853D371211C5853E388537E1
:1027240039AE51AF52E53C8E048F05FF1271CD8D49
:102734003A853C3B12123F85374175426422900131
:1027440017E0F53C753F11755904755A00AE51AF49
:1027540052E53C75F00FA4FDACF0EDD39FEC9E4028
:1027640021E53C8E048F05FF1271A2ED75F010A4D3
:10277400FFAEF0E56175F01184FD7C00ED2FF53DB1
:10278400800EE56175F01184FF7E00EF24F0F53DC5
:10279400853D37E56175F01184AFF07E008F3A1204
:1027A40011C585373EAE51AF52900117E075F00F59
:1027B400A4FDACF0EDD39FEC9E4028755904755AE6
:1027C40010853D371211C5853E38853739AE51AF76
:1027D40052E53C8E048F05FF1271CD8D3A853C3B4A
:1027E40012123F853741754264900112E0B40479B6
:1027F400900074E0FE9000E1E0D39E4037E55F7501
:10280400F00884FF7E008F37E55F75F00884ADF033
:102814007C008D3A753F08755903755A96E537C3A0
:10282400941F50051211C5800690045AE0F53785AF
:1028340037428035E55F75F00884FF7E008F37E509
:102844005F75F00884ADF07C008D3A753F087559CA
:1028540003755AB6E537C3941F50051211C5800697
:1028640090047AE0F537853742229000ABE0B4015A
:102874003BE56775F00A84FF7E008F37E56775F0E6
:102884000A84ADF07C008D3A753F0A755905755A76
:1028940012E537C3941150051211C580069005C87E
:1028A400E0F537E5422537C39464F5429000ACE087
:1028B400B4013BE56875F00A84FF7E008F37E56854
:1028C40075F00A84ADF07C008D3A753F0A755905A0
:1028D400755A7EE537C3941150051211C5800690D0
:1028E4000634E0F537E5422537C39464F542E54103
:1028F4002542F5369000B3E0B40210900907E025B4
:1029040036FE900107E0F4042EF53690010AE0D378
:1029140094014040E56BC394E7501D74E7C3956B85
:10292400FE900909E08E00F5F0E884FF7E008F3701
:10293400E5362537F536801CE56BC394E7FE900930
:1029440009E08E00F5F0E884FF7E008F37E536C39A
:102954009537F536A2034006E5412464F536E5369D
:10296400D394644009E536C39464F5368003753620
:10297400009000E3E0C3953650069000E3E0F5369E
:1029840022D200900097E0A851B800049552503E1E
:10299400900097E0A851B800049552500375360F83
:1029A400900097E004A851B800049552500375367E
:1029B40007900097E02402A851B8000495525002F1
:1029C400C200900097E060067409900075F0C22B75
:1029D4007E017F009000E9E01271B29000F8E08E71
:1029E400048F05FF1271A2E55FBC000CD39D400863
:1029F400D233740A900075F09000ABE0B4010990F2
:102A040000EAE0C39567400280159000FCE0A851FD
:102A1400B8000495525002C200740B900075F090F7
:102A240000ABE0B40107E567C394644002801D90E5
:102A34000142E0600D900142E0A851B800069552B1
:102A440040028008C200740B900075F0A20040039D
:102A5400753600C23290012BE0B4011490012CE0D1
:102A6400A851B8000495525007E55FC39560400231
:102A7400802A9000D4E0D3941D400B9000D4E0C38E
:102A8400941EF5368003753600A22F400874159005
:102A94000075F0D232D22FD22D022B7FC22DC22F3D
:102AA4009000B3E0B40306A225B3B34003022B7F26
:102AB40090090BE0C39405A851B800049552500640
:102AC400900912E06002801F9000D4E0D3941D406E
:102AD4000B9000D4E0C3941EF53680037536007461
:102AE4000C900075F0D23290090BE0A851B80004A4
:102AF40095525006900912E07002801F9000D4E0B5
:102B0400D3941D400B9000D4E0C3941EF53680038B
:102B1400753600740C900075F0D23290090BE0A861
:102B240051B80004955250319000F2E0B40228D21A
:102B34002B900911E0FE900912E0D39E50069009F3
:102B440012E070028009900911E4F0C22B80069013
:102B54000911E004F08002C20090090BE02405A8EA
:102B640051B80004955250139000F2E0B4020A9058
:102B74000912E07002D22B8002C200A22AB34027BD
:102B84009000D4E0D3941D400B9000D4E0C3941E75
:102B9400F5368003753600A22E4006741090007539
:102BA400F0D22ED2328002C22E85366C9000D4E050
:102BB400D3941D40189000A2E02536FE900074E0E6
:102BC40075F01E84FC7F00EE2CF5368037A232B3FC
:102BD40040169000A2E0FE900074E075F01E84FCA4
:102BE4007F00EE2CF536801C9000A4E02536FE9084
:102BF40000A2E02EFE900074E075F01E84FC7F00BD
:102C0400EE2CF536A233B34005D22B756C0022901E
:102C14000074E075F00584FF7E008F37900074E047
:102C240075F00584ADF07C008D3A753F0575590348
:102C3400755AD69000F6E01475F00584FF7E00E521
:102C440037BE00039F50051211C5800BE537900471
:102C54007B1271E3E0F537E53790090AF090090A31
:102C6400E0FE9000E5E0C39E50089000E5E0900986
:102C74000AF09000D4E0D3941D401E90090AE0FEAF
:102C84009000A2E02EFE900074E075F01E84FC7F9C
:102C940000EE2C90090AF0803FA232B34018900055
:102CA400A2E0FE900074E075F01E84FC7F00EE2C20
:102CB40090090AF0802290090AE0FE9000A4E02E18
:102CC400FE9000A2E02EFE900074E075F01E84FCDD
:102CD4007F00EE2C90090AF0229000ABE0B401369C
:102CE400E56775F00A84FF7E009005A5120048E0B0
:102CF400F546E546D394644010E546C3946475F004
:102D04000F84FF7E008F4680037546009000C8E064
:102D14002546F54680069000C8E0F54622E567752D
:102D2400F00A84FF7E009005A5120048E0C3946970
:102D34004007E567D394644055900112E0C39403BF
:102D440050269008A7E0FEA3E0FF7404120039E5C2
:102D54005F1271B2740F8E048F05FF1271A2900876
:102D6400A5ECF0A3EDF080249008A7E0FEA3E0FF1B
:102D74007404120039E5611271B2740F8E048F0568
:102D8400FF1271A29008A5ECF0A3EDF0800F90085B
:102D9400A7E0F8A3E09008A5C8F0A3C8F0A20340F8
:102DA4001A9008A7E0FEA3E0FF74031271B2740145
:102DB4001200399008A5EEF0A3EFF09000BBE0B448
:102DC4000262E56AC3944175F00584FF7E008F3783
:102DD400E56A75F00584ADF07C008D3A753F0575A4
:102DE4005906755A14E537C3941750051211C58056
:102DF400069006CCE0F5379008A5E0FEA3E0FF744A
:102E04000A8E048F05FF1271A2E5378C068D071216
:102E140071B2740A8E048F05FF1271A29008A5EC9A
:102E2400F0A3EDF09008A5E0FEA3E0FF9008ABE06E
:102E3400FCA3E0FDEDD39FEC9E400F9008ABE0F8BF
:102E4400A3E09008A5C8F0A3C8F022E50875F00433
:102E5400A4FFAEF09006E8120048E0903CE8F828A1
:102E64002873804C85527380479000F8E0855FF0AA
:102E7400A4FFAEF074081200398F73803385617338
:102E8400802E8567738029856873802485697380A3
:102E94001F856A73801A856B73801585667380102D
:102EA400856573800B856C738006900027E0F5734D
:103CE800022E66022E68022E6D022E81022E860298
:103CF8002E8B022E90022E95022E9A022E9F022EB5
:073D0800A4022EA9022EAE59
:102EB400E50875F004A4FFAEF09006E9120048E5B9
:102EC4000875F004A4FFAEF0E0FC9006EA12004896
:102ED400ECFEE0FFEEC39F4003022FBCE50875F053
:102EE40004A4FFAEF09006E8120048E0B40441E503
:102EF4000875F004A4FFAEF09006EA120048E0C39F
:102F04009573500AE508F50CD39234123DF9E5089F
:102F140075F004A4FFAEF09006E9120048E0D395E2
:102F240073400AE508F50CC39234123DF9022FBA36
:102F3400E50875F004A4FFAEF09006E9120048E03D
:102F4400C395735015E50875F004A4FFAEF0900620
:102F5400EA120048E0D395735002800AE508F50CA4
:102F6400D39234123DF9E50875F004A4FFAEF09055
:102F740006E9120048E0D395735015E50875F0048E
:102F8400A4FFAEF09006EA120048E0C39573500A1D
:102F9400E508F50CC39234123DF99006F0E0B40153
:102FA40009900104E0D395615002800A7402F50C83
:102FB400C39234123DF9806AE50875F004A4FFAEAB
:102FC400F09006E9120048E0D395734015E50875C2
:102FD400F004A4FFAEF09006EA120048E0C3957333
:102FE4004002800AE508F50CC39234123DF9E50865
:102FF40075F004A4FFAEF09006E9120048E0C39512
:10300400734015E50875F004A4FFAEF09006EA12CB
:103014000048E0D39573400AE508F50CD3923412C6
:103024003DF922AE2EAF2F74C9BE000CD39F4008C9
:10303400782E127205023141752F01752E00AE51A2
:10304400AF52E546BE000DD39F40099000DAE0D3AD
:10305400954740028023754700E546C39552F573B2
:103064009000DDE0D395454008E5452573F545809E
:10307400069000DDE0F545800205479000B6E0D3F8
:103084009561401CE55FC395604015AE51AF52E5B4
:1030940046BE00039F50099000DBE0D395484002F0
:1030A400806E90090CE0A851B80004955250037545
:1030B4004A0090090CE0A851B8000BD39552400681
:1030C400E55290090CF0E54A7041E552C39546F586
:1030D40073E573D3940540037573059000DCE0C376
:1030E40095455007E573C3954540028009E545C3FE
:1030F4009573F54580069000DCE0F5459000DCE032
:10310400D3954540069000DCE0F545754800800203
:103114000548E54A70169000B6E0C39561500DE588
:10312400462405A851B8000695524002800F90002D
:10313400C9E0F545754A01747890090CF022AE2E69
:10314400AF2F74E9D39F74039E4008782E12720542
:103154000232FB752F01752E00754532A226403DC3
:10316400E54775F00284AFF07E00EF4E70057545BB
:103174001980037545329000C9E075F002A4FFAED2
:10318400F0E547BE0006D39F4002D2260547754AA4
:1031940003747890090CF07549000232E2AE51AF25
:1031A40052E5466F4E70030232E2E546BE000DD38F
:1031B4009F40099000DAE0D395474002800F75479D
:1031C40000E54AC394035003754519800DE546C3D1
:1031D4009552F573E5472573F5479000B6E0D3950E
:1031E40061400E90090CE0A851B80007D3955240F5
:1031F40002800C05499000C9E0B54903754A00E511
:103204004AB40306A203B3B34002800A0549E54960
:10321400B43C03754A02E54AB4022990090CE0A8BB
:1032240051B8000ED395524009E55290090CF0753F
:1032340049009000B6E0C39561500975490074785F
:1032440090090CF0E54A705A9000B6E0D3956140BD
:103254001CE55FC395604015AE51AF52E546BE0014
:10326400039F50099000DBE0D39548400280087525
:10327400480075454B8028E552C39546F573E573C0
:10328400D3940540037573059000B6E0D39561406F
:1032940008E5482573F5488006E5482406F5487591
:1032A4004900E54A70169000B6E0C39561500DE5FB
:1032B400462405A851B80006955240028003754A79
:1032C40001E54AB4011875451905499000C9E0B5EE
:1032D4004906754A02754900747890090CF0A201F8
:1032E400B34003754532E54575F00AA4FFAEF0908E
:1032F40008B1EEF0A3EFF022E56F903D0FF8282817
:1033040073023CA89000AEE0700302362C9000E4F7
:10331400E0B4010280030234BF900072E0655E6095
:1033240009E552455160030234BC7E017F00E5BECD
:103334001271B2E5BD2FFF50010E8E598F5A9001C4
:1033440049E075F010A4FDACF08C5B8D5CEFD39D6F
:10335400EE9C40091271FD8E598F5A8006755A00F1
:10336400755900AE59AF5A740E1271B29000D9E07B
:103374008E048F05FF1271A29008B5ECF0A3EDF056
:10338400E56B600FE56BC394FE500890010AE0649E
:1033940002600280649000F8E0B40B1F9008B5E06E
:1033A400FEA3E0FF74E71271B2E56B8E048F05FF94
:1033B4001271A29008B5ECF0A3EDF09000F8E0D300
:1033C400940B40089000E0E064046002802B9008B5
:1033D400B5E0FEA3E0FF9008B9E0FCA3E0FDEFD365
:1033E4009DEE9C400D1271FD9008B5EEF0A3EFF038
:1033F40080079008B5E4F0A3F09008B5E0FEA3E0E0
:10340400FFEFD39400EE94014008D2337426900069
:1034140075F0A233B3B3502C7E057F009000F8E022
:103424008E048F05FF1271A29008B5E0FEA3E0FFA1
:10343400EFC39DEE9C400FAC51AD52740FBC000421
:10344400D39D50028002C2339000AEE0B4022790B4
:1034540008B7E0FEA3E0FF9008B5E0FCA3E0FDEFB1
:103464002DFDEE3CFC74018C068D0712003990088A
:10347400B5EEF0A3EFF09008B5E0FEA3E0FF9008EE
:10348400B7E0FCA3E0FDEDD39FEC9E4004D229807D
:1034940002B2299008B5E0F8A3E09008B7C8F0A3F9
:1034A400C8F09000E0E064016006A229B3B34002D2
:1034B40080069008B6E0F55F02362AD2297E017FA5
:1034C40000E5BE1271B2E5BD2FFF50010E8E598F7B
:1034D4005A900149E075F010A4FDACF08C5B8D5C52
:1034E400EFD39DEE9C40091271FD8E598F5A8006D0
:1034F400755A00755900AE59AF5A740E1271B290D4
:1035040000D9E08E048F05FF1271A29008B5ECF08B
:10351400A3EDF0E56B600FE56BC394FE50089001DA
:103524000AE06402600280649000F8E0B40B1F902B
:1035340008B5E0FEA3E0FF74E71271B2E56B8E04F8
:103544008F05FF1271A29008B5ECF0A3EDF0900086
:10355400F8E0D3940B40089000E0E064046002803B
:103564002B9008B5E0FEA3E0FF9008B9E0FCA3E0CF
:10357400FDEFD39DEE9C400D1271FD9008B5EEF069
:10358400A3EFF080079008B5E4F0A3F09008B5E04D
:10359400FEA3E0FFEFD39400EE94014008D233740D
:1035A40026900075F0A233B3B3502C7E057F0090B3
:1035B40000F8E08E048F05FF1271A29008B5E0FEBA
:1035C400A3E0FFEFC39DEE9C400FAC51AD52740FCE
:1035D400BC0004D39D50028002C2339000AEE0B41C
:1035E40002279008B7E0FEA3E0FF9008B5E0FCA333
:1035F400E0FDEF2DFDEE3CFC74018C068D071200FE
:10360400399008B5EEF0A3EFF09008B5E0F8A3E028
:103614009008B7C8F0A3C8F09000E0E06401600629
:103624009008B6E0F55F8003755F009000AAE07033
:1036340006756F030232FC75BB18023CA8023CA855
:103644009000AAE070030237B57E017F00E5BE1248
:1036540071B2E5BD2FFF50010E8E598F5A9000F0C4
:10366400E0B4010F7E0F7FFFAC59AD5A1271FD8E8D
:10367400598F5A900115E0B40245AE59AF5A9000E3
:1036840030E0FCA3E0FDEDD39FEC9E400A900030B7
:10369400E559F0A3E55AF0AE59AF5A900032E0FC78
:1036A400A3E0FDEFD39DEE9C400A900032E559F073
:1036B400A3E55AF0AE59AF5A74041200398F6190E1
:1036C4000115E0704CAE59AF5A900030E0FCA3E015
:1036D400FDEFD39DEE9C40091271FD8E598F5A80E7
:1036E40006755A00755900AE59AF5A74101271B26A
:1036F400900114E08E048F05FF1271A28C598D5A2B
:1037040074FFBC0009D39D4005855A61800375612F
:10371400FE9000E0E0B4010280030237B3A203B3D9
:10372400B3500E9000B4E0A851B80005D3955250A0
:103734000280719000F1E08561F0A4FFAEF0746442
:103744008E048F05FF1271A28C598D5AE56B601699
:10375400E56BC394FE500F90010AE0B40208900098
:10376400F8E0640B60028017AE59AF5A74E7127127
:10377400B2E56B8E048F05FF1271A28C598D5AAE7F
:1037840059AF5A9008B5E0FCA3E0FDEDD39FEC9E41
:103794004005855A5F800BA229B340069008B6E025
:1037A400F55F800BA229B340069008B6E0F55F8070
:1037B400037561009000ADE07006756F050232FC80
:1037C40075BB19023CA8023CA89000ADE07003024E
:1037D400389CE55ED3955D400302389A90002EE054
:1037E400FEA3E0FFE5651271F590002EEEF0A3EF65
:1037F400F090011AE0B402247E017F00E5BE12714C
:10380400B2E5BD2FFF50010E8F048E057E0F7FFFA2
:10381400CDCCCD1271FD8E598F5A80147E017F005C
:10382400E5BE1271B2E5BD2FFF50010E8E598F5ABD
:1038340090011AE07017AE59AF5A740A1271B2743B
:10384400518E048F05FF1271A28D658019AE59AF98
:103854005A740A1271B28F048E057E017F95CDCC05
:10386400CD1270A08F65E565D394644003756564DB
:1038740090002EE0FEA3E0FFE5652FFF50010E90BF
:10388400002EEEF0A3EFF09000B1E0048E048F055B
:10389400FF1271A28D6580037565329000FDE070A2
:1038A40006756F070232FC75BB13023CA8023CA8E4
:1038B4009000FDE0604A7E017F00E5BE1271B2E532
:1038C400BD2FFF50010E8E598F5A74041200398F88
:1038D400669000FFE08566F0A4FDACF07464FF120E
:1038E40071A28D669000FEE08566F0A4FFAEF074D0
:1038F400FF8E048F05FF1271A2ED900096F08003F5
:103904007566009000ABE07006756F090232FC75B5
:10391400BB17023CA8023CA89000ABE0B4010280B3
:10392400030239B07E017F00E5BE1271B2E5BD2FFE
:10393400FF50010E8E598F5A90090DE060199009BD
:103944000DE014906BF212008CE493FC740193FD6F
:10395400EDC39FEC9E4002800690090DE014F090A8
:10396400090DE0C394B3501DAE59AF5A90090DE050
:1039740004906BF212008CE493FC740193FDEFC38A
:103984009DEE9C4002800690090DE004F090090D24
:10399400E0FE9000D1E08E0088F0A4FFAEF07464E5
:1039A4008E048F05FF1271A28D67800375670090E6
:1039B40000ACE07006756F0B0232FC75BB16023C5E
:1039C400A8023CA89000ACE0B401028003023A5C77
:1039D4007E017F00E5BE1271B2E5BD2FFF50010EDE
:1039E4008E598F5A90090EE0601990090EE01490D8
:1039F4006D5C12008CE493FC740193FDEDC39FECA9
:103A04009E4002800690090EE014F090090EE0C377
:103A140094B3501DAE59AF5A90090EE004906D5CFA
:103A240012008CE493FC740193FDEFC39DEE9C4063
:103A340002800690090EE004F090090EE0FE90006A
:103A4400D7E08E0088F0A4FFAEF074648E048F0576
:103A5400FF1271A28D68800375680075BB1F023C5C
:103A6400A8023CA87E017F00E5BE1271B2E5BD2F1D
:103A7400FF50010E8E598F5A74091271B274E68E7A
:103A8400048F05FF1271A28D6A9000B3E070067571
:103A94006F0F0232FC75BB15023CA8023CA89000D3
:103AA400B3E07003023BF37E017F00E5BE1271B206
:103AB400E5BD2FFF50010E8E598F5A740412003940
:103AC4008F699000B3E0B40115900107E08569F0B7
:103AD400A4FFAEF07407120039EF900908F09000CB
:103AE400B3E0B40215900107E08569F0A4FFAEF0DD
:103AF4007407120039EF900907F09000B3E0B403A3
:103B0400028003023BD69000F4E07052E569C3944E
:103B140019500FD2259000D3E090090BF0900910B2
:103B2400E4F0E569D394644004A2254002802D901A
:103B34000910E004F0900910E0FE900146E0B5069B
:103B44000B90090BE004F0900910E4F090090BE0ED
:103B540064966006900146E07002C225806390007E
:103B6400D3E07034900107E08569F0A4FFAEF074EF
:103B7400FF8E048F05FF1271A2ED90090BF0AE5178
:103B8400AF52741EBE0006D39F4002D225E561D316
:103B940094E54002C2258029E569C3940A500DAE1C
:103BA40051AF52741EBE0004D39F50028002D2252E
:103BB400E561D394E54002C2259000D3E090090B5F
:103BC400F090090BE0C394055006740590090BF0BE
:103BD400C22A9000B3E0B40414E569C394195002F6
:103BE400D22AE569D394324002C22AC225800375E1
:103BF400690090010AE07006756F110232FC75BB12
:103C040014023CA8023CA890010AE07003023C950F
:103C14007E017F00E5BE1271B2E5BD2FFF50010E9B
:103C24008E598F5A90014AE075F010A4FDACF08CC7
:103C34005B8D5CEFD39DEE9C40091271FD8E598F14
:103C44005A8006755A00755900AE59AF5A740E124F
:103C540071B2900111E08E048F05FF1271A28C5B8A
:103C64008D5C74FFBC00039D5005756BFF8003855C
:103C74005C6BE56B75F00BA4FFAEF09000F8E08E82
:103C8400048F05FF1271A29008B9ECF0A3EDF08047
:103C940003756B009000AEE0600575BB1A80037578
:043CA400BB188000C9
:103D0F000233050233080236410236440237CA0233
:103D1F0037CD0238B10238B402391902391C0239D1
:103D2F00C50239C8023A65023A68023A9F023AA2BE
:093D3F00023C08023C0B023CA806
:103CA800E56F75F00284AFF07E00EF4E7002D2EC43
:033CB800056F2273
:0971E3002582F582500205832289
:0F008C0025E050020583258250020583F582226C
:10718100EF2F500205832582F582E5833E2EF5839C
:0171910022DB
:1071F500CFC39FFF50011E22C3EF9DFFEE9CFE22D1
:087205000806B600021806227B
:0D71C000A3E004F070061271D9E004F02283
:0E003900048007C3CE13CECF13CFD5E0F6223E
:1070A000BC000FBE0008ED8FF084FFADF022E4FEBF
:1070B000FF22BE000DEF60FE54F0606F20E7030278
:1070C0007156EAC0E0EBC0E078017A0075F001EE9D
:1070D00020E710EF25E0FFEE33FE0AC5F023C5F0F0
:1070E00030E7F0EA5407F9096A7A007B006001088A
:1070F000C3EC9E40167004ED9F4010ED9FFDEC9E8A
:10710000FCE5F0CA4ACA03F5F08005E5F003F5F0A6
:10711000C3EE13FEEF13FFD9D77908CACBCAD8D074
:10712000EAFEEBFFD0E0FBD0E0FA22EC8FF084FC2B
:10713000ED54F045F0C48FF084FEEDC454F045F0FA
:10714000C48FF084FDEEC4FE54F02DFFEE540F3CCE
:10715000FEADF07C0022790078008FF0EC7E0820F4
:10716000E70DC3CD33CD33C933C9C833C8DEF0848E
:1071700049F9E5F08FF0BE00E6FD7C00E9FFE8FE8E
:0171800022EC
:0E71B200F88FF0A4FFE5F0CE88F0A42EFE22A8
:10000300EF8DF0A4F9A8F0EF8CF0A428F8EE8DF0B2
:06001300A428FEE9FF2213
:10719200600D782B02719C007830D8FED5E0F82281
:1071A200EEC0E07E001270A0EFFDEEFCD0E0FE2209
:0C71CD00EEC0E07E001270A0D0E0FE22B8
:03001B0002001EC2
:0300530002005652
:03009B00020071EF
:030000000271EC9E
:0971EC0075817575D000024AE5B9
:0B004800E5822FF582E5833EF5832260
:0A71D9000582D5820215831582227B
:10001E00C0E0C0F0C083C082C0D075D000124A8943
:0B002E00D0D0D082D083D0F0D0E032E0
:10005600C0E0C0F0C083C082C0D075D000124A8C08
:10006600D0D0D082D083D0F0D0E032C0E0C0F0C093
:1000760083C082C0D075D000124AAED0D0D082D014
:0600860083D0F0D0E0324F
:00000001FF
